 KbdUs

 Timestamp is 4da2a513 (Mon Apr 11 18:52:03 2011)

 Preferred load address is 10000000

 Start         Length     Name                   Class
 0001:00000000 00000004H .CRT$XCA                CODE
 0001:00000004 00000004H .CRT$XCZ                CODE
 0001:00000008 00000004H .CRT$XIA                CODE
 0001:0000000c 00000004H .CRT$XIZ                CODE
 0001:00000010 00000004H .CRT$XPA                CODE
 0001:00000014 00000004H .CRT$XPZ                CODE
 0001:00000018 00000004H .CRT$XTA                CODE
 0001:0000001c 00000004H .CRT$XTZ                CODE
 0001:00000020 000039beH .rdata                  CODE
 0001:000039e0 00000022H .rdata$debug            CODE
 0001:00003a04 0000db50H .text                   CODE
 0001:00011554 000000c8H .xdata                  CODE
 0001:0001161c 0000003cH .idata$2                CODE
 0001:00011658 00000014H .idata$3                CODE
 0001:0001166c 00000130H .idata$4                CODE
 0001:0001179c 0000007eH .idata$6                CODE
 0001:00011820 00000232H .edata                  CODE
 0002:00000000 00000130H .idata$5                DATA
 0002:00000130 00000880H .data                   DATA
 0002:000009b0 000004c4H .bss                    DATA
 0003:00000000 00000450H .pdata                  DATA

  Address         Publics by Value              Rva+Base       Lib:Object

 0000:00000000       ___safe_se_handler_table   00000000     <absolute>
 0000:00000000       ___safe_se_handler_count   00000000     <absolute>
 0001:00000000       __xc_a                     10001000     corelib0:crt0init.obj
 0001:00000004       __xc_z                     10001004     corelib0:crt0init.obj
 0001:00000008       __xi_a                     10001008     corelib0:crt0init.obj
 0001:0000000c       __xi_z                     1000100c     corelib0:crt0init.obj
 0001:00000010       __xp_a                     10001010     corelib0:crt0init.obj
 0001:00000014       __xp_z                     10001014     corelib0:crt0init.obj
 0001:00000018       __xt_a                     10001018     corelib0:crt0init.obj
 0001:0000001c       __xt_z                     1000101c     corelib0:crt0init.obj
 0001:00000040       ??_C@_1FE@DBIINFNI@?$AAK?$AAP?$AAP?$AAL?$AAa?$AAy?$AAo?$AAu?$AAt?$AA?3?$AA?5?$AAd?$AAa?$AAt?$AAa?$AA?5?$AAs?$AAt?$AAr?$AAu?$AAc?$AAt?$AAu?$AAr?$AAe?$AA?5?$AAs?$AAi?$AAz?$AAe?$AA?5?$AAm@ 10001040     BSPKeypad:bspkeypad.obj
 0001:00000098       ??_C@_1FK@FNONLNGN@?$AA?$CF?$AAs?$AA?3?$AA?5?$AAD?$AAE?$AAB?$AAU?$AAG?$AAC?$AAH?$AAK?$AA?5?$AAf?$AAa?$AAi?$AAl?$AAe?$AAd?$AA?5?$AAi?$AAn?$AA?5?$AAf?$AAi?$AAl?$AAe?$AA?5?$AA?$CF?$AAs?$AA?5?$AAa@ 10001098     BSPKeypad:bspkeypad.obj
 0001:000000f8       ??_C@_1KG@FMLIDDK@?$AAc?$AA?3?$AA?2?$AAw?$AAi?$AAn?$AAc?$AAe?$AAr?$AAo?$AAo?$AAt?$AAs?$AA?2?$AAt?$AAo?$AAp?$AAa?$AAz?$AA?2?$AAw?$AAi?$AAn?$AAc?$AAe?$AA7?$AA0?$AA0?$AA?2?$AAp?$AAl?$AAa@ 100010f8     BSPKeypad:bspkeypad.obj
 0001:000001a0       ??_C@_1O@IKMMPJPA@?$AA?9?$AA?9?$AA?$CF?$AAs?$AA?$AN?$AA?6?$AA?$AA@ 100011a0     BSPKeypad:bspkeypad.obj
 0001:000001b0       ??_C@_1II@EMPIEEJ@?$AAE?$AAn?$AAd?$AA?5?$AAo?$AAf?$AA?5?$AAI?$AAn?$AAi?$AAt?$AA?5?$AAm?$AAe?$AAt?$AAh?$AAo?$AAd?$AA?5?$AA?9?$AA?5?$AAc?$AAt?$AAr?$AAl?$AA?3?$AA?5?$AA?$CF?$AAx?$AA?5?$AA?5?$AAs@ 100011b0     BSPKeypad:bspkeypad.obj
 0001:00000238       ??_C@_1DA@LMIFJCLG@?$AA?$FL?$AAK?$AAP?$AAP?$AA?$FN?$AA?$CF?$AAs?$AA?3?$AA?5?$AA?5?$AAg?$AA_?$AAp?$AAK?$AAP?$AAP?$AA?$DN?$AA0?$AAx?$AA?$CF?$AAx?$AA?$AN?$AA?6?$AA?$AA@ 10001238     BSPKeypad:bspkeypad.obj
 0001:00000268       ??_C@_1EO@MCAICMBL@?$AA?$CF?$AAs?$AA?3?$AA?5?$AAK?$AAP?$AAP?$AA?5?$AAm?$AAe?$AAm?$AAo?$AAr?$AAy?$AA?5?$AAs?$AAp?$AAa?$AAc?$AAe?$AA?5?$AAm?$AAa?$AAp?$AAp?$AAi?$AAn?$AAg?$AA?5?$AAf?$AAa?$AAi@ 10001268     BSPKeypad:bspkeypad.obj
 0001:000002b8       ??_C@_1O@JNDDBHKG@?$AA?$CL?$AA?$CL?$AA?$CF?$AAs?$AA?$AN?$AA?6?$AA?$AA@ 100012b8     BSPKeypad:bspkeypad.obj
 0001:000002c8       ??_C@_1BM@OPAJHIMO@?$AAB?$AAS?$AAP?$AAK?$AAp?$AAp?$AAR?$AAe?$AAg?$AAI?$AAn?$AAi?$AAt?$AA?$AA@ 100012c8     BSPKeypad:bspkeypad.obj
 0001:000002e4       ??_C@_1CG@HGHEHNPB@?$AAB?$AAS?$AAP?$AAK?$AAP?$AAP?$AAG?$AAe?$AAt?$AAS?$AAc?$AAa?$AAn?$AAC?$AAo?$AAd?$AAe?$AAs?$AA?$AA@ 100012e4     BSPKeypad:bspkeypad.obj
 0001:0000030c       ??_C@_1DE@KHLKCBMI@?$AAS?$AAc?$AAa?$AAn?$AA?5?$AAs?$AAe?$AAq?$AAu?$AAe?$AAn?$AAc?$AAe?$AA?5?$AAc?$AAo?$AAm?$AAp?$AAl?$AAe?$AAt?$AAe?$AAd?$AA?$AN?$AA?6?$AA?$AA@ 1000130c     BSPKeypad:bspkeypad.obj
 0001:00000340       ??_C@_1DK@HBNBGJO@?$AAK?$AAe?$AAy?$AAs?$AA?5?$AAd?$AAe?$AAp?$AAr?$AAe?$AAs?$AAs?$AAe?$AAd?$AA?5?$AA?$DM?$AA?5?$AA1?$AA?5?$AAp?$AAe?$AAr?$AAi?$AAo?$AAd?$AA?4?$AA?$AN?$AA?6?$AA?$AA@ 10001340     BSPKeypad:bspkeypad.obj
 0001:00000380       ??_C@_1EG@BNNCCNDO@?$AAR?$AAe?$AAl?$AAe?$AAa?$AAs?$AAe?$AA?5?$AAi?$AAn?$AAt?$AAe?$AAr?$AAr?$AAu?$AAp?$AAt?$AA?0?$AA?5?$AAK?$AAP?$AAS?$AAR?$AA?5?$AA0?$AAx?$AA?$CF?$AA0?$AA4?$AAx?$AA?4?$AA?5@ 10001380     BSPKeypad:bspkeypad.obj
 0001:000003c8       ??_C@_1CO@CDKOJIEH@?$AAK?$AAe?$AAy?$AAp?$AAr?$AAe?$AAs?$AAs?$AA?5?$AAd?$AAe?$AAb?$AAo?$AAu?$AAn?$AAc?$AAe?$AAd?$AA?4?$AA?5?$AA?$AN?$AA?6?$AA?$AA@ 100013c8     BSPKeypad:bspkeypad.obj
 0001:000003f8       ??_C@_1FM@GDGFDNMF@?$AAK?$AAe?$AAy?$AA?5?$AAp?$AAr?$AAe?$AAs?$AAs?$AAe?$AAd?$AA?0?$AA?5?$AAt?$AAe?$AAm?$AAp?$AAK?$AAP?$AAS?$AAR?$AA?5?$AA0?$AAx?$AA?$CF?$AA0?$AA4?$AAx?$AA?0?$AA?5?$AAK?$AAP@ 100013f8     BSPKeypad:bspkeypad.obj
 0001:00000458       ??_C@_1FO@LAOFEAMO@?$AAK?$AAe?$AAy?$AA?5?$AAr?$AAe?$AAl?$AAe?$AAa?$AAs?$AAe?$AAd?$AA?0?$AA?5?$AAt?$AAe?$AAm?$AAp?$AAK?$AAP?$AAS?$AAR?$AA?5?$AA0?$AAx?$AA?$CF?$AA0?$AA4?$AAx?$AA?0?$AA?5?$AAK@ 10001458     BSPKeypad:bspkeypad.obj
 0001:000004b8       ??_C@_1EC@GCKBKDBM@?$AAC?$AAh?$AAa?$AAn?$AAg?$AAe?$AAd?$AA?3?$AA?5?$AAd?$AAe?$AAp?$AAr?$AAe?$AAs?$AAs?$AAe?$AAd?$AA?5?$AA?$DM?$AA?5?$AA1?$AA?5?$AAp?$AAe?$AAr?$AAi?$AAo?$AAd?$AA?4?$AA?$AN?$AA?6@ 100014b8     BSPKeypad:bspkeypad.obj
 0001:00000500       ??_C@_1EG@DODJEDOI@?$AAD?$AAe?$AAp?$AAr?$AAe?$AAs?$AAs?$AA?5?$AAi?$AAn?$AAt?$AAe?$AAr?$AAr?$AAu?$AAp?$AAt?$AA?0?$AA?5?$AAK?$AAP?$AAS?$AAR?$AA?5?$AA0?$AAx?$AA?$CF?$AA0?$AA4?$AAx?$AA?4?$AA?5@ 10001500     BSPKeypad:bspkeypad.obj
 0001:00000548       ??_C@_1FM@PDOELOIJ@?$AAB?$AAe?$AAf?$AAo?$AAr?$AAe?$AA?5?$AAs?$AAc?$AAa?$AAn?$AA?0?$AA?5?$AAt?$AAe?$AAm?$AAp?$AAK?$AAP?$AAS?$AAR?$AA?5?$AA0?$AAx?$AA?$CF?$AA0?$AA4?$AAx?$AA?0?$AA?5?$AAK?$AAP@ 10001548     BSPKeypad:bspkeypad.obj
 0001:000005a4       ??_C@_1CA@IJDBLKLM@?$AAK?$AAp?$AAp?$AAS?$AAc?$AAa?$AAn?$AAS?$AAe?$AAq?$AAu?$AAe?$AAn?$AAc?$AAe?$AA?$AA@ 100015a4     BSPKeypad:bspkeypad.obj
 0001:000005c4       ??_C@_1BM@CGKCPMCA@?$AAB?$AAS?$AAP?$AAK?$AAp?$AAp?$AAP?$AAo?$AAw?$AAe?$AAr?$AAO?$AAn?$AA?$AA@ 100015c4     BSPKeypad:bspkeypad.obj
 0001:000005e0       ??_C@_1BO@NDJBJGIF@?$AAB?$AAS?$AAP?$AAK?$AAp?$AAp?$AAP?$AAo?$AAw?$AAe?$AAr?$AAO?$AAf?$AAf?$AA?$AA@ 100015e0     BSPKeypad:bspkeypad.obj
 0001:00000600       ??_C@_1FG@GMGPANNE@?$AA?$CF?$AAs?$AA?3?$AA?5?$AAF?$AAa?$AAi?$AAl?$AAe?$AAd?$AA?5?$AAt?$AAo?$AA?5?$AAs?$AAe?$AAt?$AA?5?$AAC?$AAR?$AAM?$AA?5?$AAc?$AAl?$AAo?$AAc?$AAk?$AA?5?$AAg?$AAa?$AAt?$AAi@ 10001600     BSPKeypad:bspkeypad.obj
 0001:00000658       ??_C@_1DC@GPJMDOPB@?$AAB?$AAS?$AAP?$AAK?$AAp?$AAp?$AAS?$AAe?$AAt?$AAC?$AAl?$AAo?$AAc?$AAk?$AAG?$AAa?$AAt?$AAi?$AAn?$AAg?$AAM?$AAo?$AAd?$AAe?$AA?$AA@ 10001658     BSPKeypad:bspkeypad.obj
 0001:00000890       ??_C@_1DO@NOHFLPBO@?$AAD?$AAa?$AAt?$AAa?$AA?5?$AAs?$AAt?$AAr?$AAu?$AAc?$AAt?$AAu?$AAr?$AAe?$AA?5?$AAs?$AAi?$AAz?$AAe?$AA?5?$AAm?$AAi?$AAs?$AAm?$AAa?$AAt?$AAc?$AAh?$AA?$AN?$AA?6?$AA?$AA@ 10001890     InputLang_0409:IL_0409.obj
 0001:000008d0       ??_C@_1CI@OHCJFJPM@?$AAE?$AAR?$AAR?$AAO?$AAR?$AA?3?$AA?5?$AA?$CF?$AAs?$AA?5?$AAl?$AAi?$AAn?$AAe?$AA?5?$AA?$CF?$AAd?$AA?3?$AA?5?$AA?$AA@ 100018d0     InputLang_0409:IL_0409.obj
 0001:000008f8       ??_C@_1BA@LEPJIIOK@?$AAU?$AAn?$AAk?$AAn?$AAo?$AAw?$AAn?$AA?$AA@ 100018f8     InputLang_0409:IL_0409.obj
 0001:00000908       ??_C@_1JE@PHGDCMNK@?$AAd?$AA?3?$AA?2?$AAc?$AAh?$AAe?$AAl?$AAa?$AAn?$AAr?$AAt?$AAm?$AA2?$AA?2?$AAp?$AAu?$AAb?$AAl?$AAi?$AAc?$AA?2?$AAc?$AAo?$AAm?$AAm?$AAo?$AAn?$AA?2?$AAo?$AAa?$AAk?$AA?2@ 10001908     InputLang_0409:IL_0409.obj
 0001:00000ac0       ??_C@_1IA@FHNGCBDJ@?$AAd?$AA?3?$AA?2?$AAc?$AAh?$AAe?$AAl?$AAa?$AAn?$AAr?$AAt?$AAm?$AA2?$AA?2?$AAp?$AAu?$AAb?$AAl?$AAi?$AAc?$AA?2?$AAc?$AAo?$AAm?$AAm?$AAo?$AAn?$AA?2?$AAo?$AAa?$AAk?$AA?2@ 10001ac0     LayoutManager:LayMgr.obj
 0001:00000b40       ??_C@_1EO@EPMBOPPE@?$AA?$CF?$AAs?$AA?3?$AA?5?$AAM?$AAa?$AAp?$AAp?$AAe?$AAd?$AA?5?$AAv?$AAk?$AAe?$AAy?$AA?5?$AA?$CF?$AA0?$AA2?$AAx?$AA?5?$AAt?$AAo?$AA?5?$AAc?$AAh?$AAa?$AAr?$AA?5?$AA?$CF?$AA0?$AA4@ 10001b40     LayoutManager:LayMgr.obj
 0001:00000b90       ??_C@_1FC@OFDMNFOP@?$AA?$CF?$AAs?$AA?3?$AA?5?$AAC?$AAh?$AAa?$AAn?$AAg?$AAi?$AAn?$AAg?$AA?5?$AAl?$AAi?$AAg?$AAh?$AAt?$AA?5?$AAs?$AAt?$AAa?$AAt?$AAe?$AA?5?$AAf?$AAo?$AAr?$AA?5?$AAV?$AAK?$AAe@ 10001b90     LayoutManager:LayMgr.obj
 0001:00000be8       ??_C@_1HA@EHIGJNFN@?$AAK?$AAe?$AAy?$AAb?$AAd?$AAD?$AAr?$AAi?$AAv?$AAe?$AAr?$AAV?$AAK?$AAe?$AAy?$AAT?$AAo?$AAU?$AAn?$AAi?$AAc?$AAo?$AAd?$AAe?$AA?3?$AA?5?$AAN?$AAo?$AA?5?$AAi?$AAn?$AAp@ 10001be8     LayoutManager:LayMgr.obj
 0001:00000c58       ??_C@_1DC@PMCHLMJK@?$AAK?$AAe?$AAy?$AAb?$AAd?$AAD?$AAr?$AAi?$AAv?$AAe?$AAr?$AAV?$AAK?$AAe?$AAy?$AAT?$AAo?$AAU?$AAn?$AAi?$AAc?$AAo?$AAd?$AAe?$AA?$AA@ 10001c58     LayoutManager:LayMgr.obj
 0001:00000c90       ??_C@_1GA@OJOBFCAJ@?$AAV?$AAa?$AAl?$AAi?$AAd?$AAa?$AAt?$AAe?$AAI?$AAn?$AAp?$AAu?$AAt?$AAL?$AAa?$AAn?$AAg?$AAu?$AAa?$AAg?$AAe?$AA?3?$AA?5?$AAI?$AAn?$AAv?$AAa?$AAl?$AAi?$AAd?$AA?5?$AAi@ 10001c90     LayoutManager:LayMgr.obj
 0001:00000cf0       ??_C@_1DG@HEJMDLH@?$AA?$CF?$AAs?$AA?3?$AA?5?$AAN?$AAe?$AAw?$AA?5?$AAd?$AAe?$AAa?$AAd?$AA?5?$AAc?$AAh?$AAa?$AAr?$AA?5?$AA0?$AAx?$AA?$CF?$AA0?$AA4?$AAx?$AA?$AN?$AA?6?$AA?$AA@ 10001cf0     LayoutManager:LayMgr.obj
 0001:00000d28       ??_C@_1BM@FJHJIGLC@?$AAG?$AAe?$AAt?$AAC?$AAh?$AAa?$AAr?$AAa?$AAc?$AAt?$AAe?$AAr?$AAs?$AA?$AA@ 10001d28     LayoutManager:LayMgr.obj
 0001:00000d48       ??_C@_1KA@IKFNAPIN@?$AAW?$AAr?$AAi?$AAt?$AAe?$AAT?$AAo?$AAC?$AAh?$AAa?$AAr?$AAB?$AAu?$AAf?$AAf?$AAe?$AAr?$AA?3?$AA?5?$AAC?$AAh?$AAa?$AAr?$AAa?$AAc?$AAt?$AAe?$AAr?$AA?5?$AAb?$AAu?$AAf@ 10001d48     LayoutManager:LayMgr.obj
 0001:00000de8       ??_C@_1EG@JFLKDNHK@?$AA?$CF?$AAs?$AA?3?$AA?5?$AAN?$AAo?$AA?5?$AAs?$AAu?$AAp?$AAp?$AAo?$AAr?$AAt?$AA?5?$AAf?$AAo?$AAr?$AA?5?$AAD?$AAK?$AAF?$AA_?$AAD?$AAE?$AAA?$AAD?$AA?5?$AAf?$AAl?$AAa?$AAg@ 10001de8     LayoutManager:LayMgr.obj
 0001:00000e30       ??_C@_1CA@HFJCLOBN@?$AAP?$AAr?$AAo?$AAc?$AAe?$AAs?$AAs?$AAD?$AAe?$AAa?$AAd?$AAK?$AAe?$AAy?$AAs?$AA?$AA@ 10001e30     LayoutManager:LayMgr.obj
 0001:00000e50       ??_C@_1HE@OBOBMNCE@?$AA?$CF?$AAs?$AA?3?$AA?5?$AAD?$AAe?$AAa?$AAd?$AA?5?$AAk?$AAe?$AAy?$AA?5?$AA?$CL?$AA?5?$AAl?$AAi?$AAg?$AAa?$AAt?$AAu?$AAr?$AAe?$AA?5?$AA0?$AAx?$AA?$CF?$AA0?$AA4?$AAx?$AA?5?$AAp@ 10001e50     LayoutManager:LayMgr.obj
 0001:00000ec8       ??_C@_1GE@GJAGNIFN@?$AAP?$AAr?$AAo?$AAc?$AAe?$AAs?$AAs?$AAL?$AAi?$AAg?$AAa?$AAt?$AAu?$AAr?$AAe?$AA?3?$AA?5?$AAT?$AAo?$AAo?$AA?5?$AAm?$AAa?$AAn?$AAy?$AA?5?$AAc?$AAh?$AAa?$AAr?$AAa?$AAc@ 10001ec8     LayoutManager:LayMgr.obj
 0001:00000f30       ??_C@_1GE@EEKLGEPK@?$AAP?$AAr?$AAo?$AAc?$AAe?$AAs?$AAs?$AAL?$AAi?$AAg?$AAa?$AAt?$AAu?$AAr?$AAe?$AA?3?$AA?5?$AAW?$AAC?$AAH?$AA_?$AAL?$AAG?$AAT?$AAR?$AA?5?$AAb?$AAu?$AAt?$AA?5?$AAn?$AAo@ 10001f30     LayoutManager:LayMgr.obj
 0001:00000f94       ??_C@_1CA@FPHGOPGB@?$AAP?$AAr?$AAo?$AAc?$AAe?$AAs?$AAs?$AAL?$AAi?$AAg?$AAa?$AAt?$AAu?$AAr?$AAe?$AA?$AA@ 10001f94     LayoutManager:LayMgr.obj
 0001:00000fb8       ??_C@_1FI@LMKMPEMM@?$AAM?$AAa?$AAp?$AAV?$AAi?$AAr?$AAt?$AAu?$AAa?$AAl?$AAK?$AAe?$AAy?$AA?3?$AA?5?$AAN?$AAo?$AA?5?$AAd?$AAe?$AAv?$AAi?$AAc?$AAe?$AA?5?$AAl?$AAa?$AAy?$AAo?$AAu?$AAt?$AA?5@ 10001fb8     LayoutManager:LayMgr.obj
 0001:00001010       ??_C@_1FK@KLIIDPFG@?$AAM?$AAa?$AAp?$AAV?$AAi?$AAr?$AAt?$AAu?$AAa?$AAl?$AAK?$AAe?$AAy?$AA?3?$AA?5?$AAN?$AAo?$AA?5?$AAi?$AAn?$AAp?$AAu?$AAt?$AA?5?$AAl?$AAa?$AAn?$AAg?$AAu?$AAa?$AAg?$AAe@ 10002010     LayoutManager:LayMgr.obj
 0001:00001070       ??_C@_1GK@PNFGDIJE@?$AA?$CF?$AAs?$AA?3?$AA?5?$AAL?$AAa?$AAy?$AAo?$AAu?$AAt?$AA?5?$AAM?$AAa?$AAn?$AAa?$AAg?$AAe?$AAr?$AA?5?$AAs?$AAu?$AAc?$AAc?$AAe?$AAs?$AAs?$AAf?$AAu?$AAl?$AAl?$AAy?$AA?5@ 10002070     LayoutManager:LayMgr.obj
 0001:000010e0       ??_C@_1GK@EADJFIFB@?$AAK?$AAe?$AAy?$AAb?$AAo?$AAa?$AAr?$AAd?$AA?3?$AA?5?$AAE?$AAr?$AAr?$AAo?$AAr?$AA?5?$AAs?$AAe?$AAl?$AAe?$AAc?$AAt?$AAi?$AAn?$AAg?$AA?5?$AAd?$AAe?$AAv?$AAi?$AAc?$AAe@ 100020e0     LayoutManager:LayMgr.obj
 0001:00001150       ??_C@_1ME@GIAPPCNP@?$AAK?$AAe?$AAy?$AAb?$AAo?$AAa?$AAr?$AAd?$AA?3?$AA?5?$AAC?$AAo?$AAu?$AAl?$AAd?$AA?5?$AAn?$AAo?$AAt?$AA?5?$AAa?$AAc?$AAt?$AAi?$AAv?$AAa?$AAt?$AAe?$AA?5?$AAt?$AAh?$AAe@ 10002150     LayoutManager:LayMgr.obj
 0001:00001218       ??_C@_1EI@JGJOLDCK@?$AA?$CF?$AAs?$AA?3?$AA?5?$AAF?$AAo?$AAu?$AAn?$AAd?$AA?5?$AAd?$AAe?$AAf?$AAa?$AAu?$AAl?$AAt?$AA?5?$AAi?$AAn?$AAp?$AAu?$AAt?$AA?5?$AAm?$AAe?$AAt?$AAh?$AAo?$AAd?$AA?5?$AA?$CF@ 10002218     LayoutManager:LayMgr.obj
 0001:00001260       ??_C@_1LE@PONPAOJG@?$AAK?$AAe?$AAy?$AAb?$AAo?$AAa?$AAr?$AAd?$AA?3?$AA?5?$AAD?$AAe?$AAf?$AAa?$AAu?$AAl?$AAt?$AA?5?$AAi?$AAn?$AAp?$AAu?$AAt?$AA?5?$AAm?$AAe?$AAt?$AAh?$AAo?$AAd?$AA?5?$AAs@ 10002260     LayoutManager:LayMgr.obj
 0001:00001314       ??_C@_11LOCGONAA@?$AA?$AA@ 10002314     LayoutManager:LayMgr.obj
 0001:00001318       ??_C@_1FA@LOAOONFK@?$AA?$CF?$AAs?$AA?3?$AA?5?$AAI?$AAn?$AAi?$AAt?$AAi?$AAa?$AAl?$AAi?$AAz?$AAe?$AAd?$AA?5?$AAP?$AAD?$AAD?$AA?5?$AA?$CF?$AAu?$AA?5?$AA?9?$AA?5?$AA?$CF?$AAs?$AA?5?$AA?$CI?$AAM?$AAa?$AAs@ 10002318     LayoutManager:LayMgr.obj
 0001:00001368       ??_C@_1BAK@OADNNFLN@?$AAK?$AAe?$AAy?$AAb?$AAo?$AAa?$AAr?$AAd?$AA?3?$AA?5?$AA?8?$AA?$CF?$AAs?$AA?8?$AA?5?$AAd?$AAi?$AAd?$AA?5?$AAn?$AAo?$AAt?$AA?5?$AAc?$AAa?$AAl?$AAl?$AA?5?$AAK?$AAe?$AAy?$AAb@ 10002368     LayoutManager:LayMgr.obj
 0001:00001478       ??_C@_1GK@CFECEMAO@?$AAK?$AAe?$AAy?$AAb?$AAo?$AAa?$AAr?$AAd?$AA?3?$AA?5?$AAI?$AAn?$AAv?$AAa?$AAl?$AAi?$AAd?$AA?5?$AAk?$AAe?$AAy?$AAb?$AAd?$AA?5?$AAP?$AAD?$AAD?$AA?5?$AAi?$AAn?$AAf?$AAo@ 10002478     LayoutManager:LayMgr.obj
 0001:000014e8       ??_C@_1FC@BFKJMBD@?$AAK?$AAe?$AAy?$AAb?$AAo?$AAa?$AAr?$AAd?$AA?3?$AA?5?$AAP?$AAD?$AAD?$AA?5?$AA?$CF?$AAu?$AA?5?$AAi?$AAn?$AAi?$AAt?$AAi?$AAa?$AAl?$AAi?$AAz?$AAa?$AAt?$AAi?$AAo?$AAn?$AA?5@ 100024e8     LayoutManager:LayMgr.obj
 0001:0000153c       ??_C@_1CA@PAEAFIKJ@?$AAO?$AAu?$AAt?$AA?5?$AAo?$AAf?$AA?5?$AAm?$AAe?$AAm?$AAo?$AAr?$AAy?$AA?$AN?$AA?6?$AA?$AA@ 1000253c     LayoutManager:LayMgr.obj
 0001:00001560       ??_C@_1FG@KKEHCAMF@?$AAU?$AAn?$AAa?$AAb?$AAl?$AAe?$AA?5?$AAt?$AAo?$AA?5?$AAs?$AAe?$AAt?$AA?5?$AAu?$AAp?$AA?5?$AAk?$AAe?$AAy?$AAb?$AAo?$AAa?$AAr?$AAd?$AA?5?$AAl?$AAa?$AAy?$AAo?$AAu?$AAt@ 10002560     LayoutManager:LayMgr.obj
 0001:000015b8       ??_C@_1DA@ENNNKOKA@?$AAK?$AAe?$AAy?$AAb?$AAd?$AAD?$AAr?$AAi?$AAv?$AAe?$AAr?$AAI?$AAn?$AAi?$AAt?$AAi?$AAa?$AAl?$AAi?$AAz?$AAe?$AAE?$AAx?$AA?$AA@ 100025b8     LayoutManager:LayMgr.obj
 0001:000015e8       ??_C@_1EK@HNKEACEC@?$AAK?$AAe?$AAy?$AAb?$AAo?$AAa?$AAr?$AAd?$AA?5?$AAe?$AAv?$AAe?$AAn?$AAt?$AA?5?$AAt?$AAh?$AAr?$AAe?$AAa?$AAd?$AA?5?$AAt?$AAe?$AAr?$AAm?$AAi?$AAn?$AAa?$AAt?$AAi?$AAn@ 100025e8     LayoutManager:LayMgr.obj
 0001:00001638       ??_C@_1IO@FAAGELJD@?$AA?$CF?$AAs?$AA?3?$AA?5?$AAP?$AAD?$AAD?$AA?5?$AA?$CF?$AAu?$AA?3?$AA?5?$AAS?$AAc?$AAa?$AAn?$AA?5?$AAc?$AAo?$AAd?$AAe?$AA?5?$AA0?$AAx?$AA?$CF?$AA0?$AA8?$AAx?$AA?5?$AA?9?$AA?$DO?$AA?5@ 10002638     LayoutManager:LayMgr.obj
 0001:000016c8       ??_C@_1HE@NMPGFJEM@?$AA?$CF?$AAs?$AA?3?$AA?5?$AAP?$AAD?$AAD?$AA?5?$AA?$CF?$AAu?$AA?3?$AA?5?$AAU?$AAs?$AAi?$AAn?$AAg?$AA?5?$AAd?$AAe?$AAv?$AAi?$AAc?$AAe?$AA?5?$AAl?$AAa?$AAy?$AAo?$AAu?$AAt?$AA?5@ 100026c8     LayoutManager:LayMgr.obj
 0001:00001740       ??_C@_1EG@GJMMGGFM@?$AA?$CF?$AAs?$AA?3?$AA?5?$AAk?$AAe?$AAy?$AAb?$AAd?$AA?5?$AA?$CF?$AAu?$AA?5?$AAs?$AAc?$AAa?$AAn?$AA?5?$AAc?$AAo?$AAd?$AAe?$AA?5?$AA0?$AAx?$AA?$CF?$AA0?$AA8?$AAx?$AA?7?$AA?$CF?$AAs@ 10002740     LayoutManager:LayMgr.obj
 0001:00001788       ??_C@_19EPDBDPAN@?$AAD?$AAo?$AAw?$AAn?$AA?$AA@ 10002788     LayoutManager:LayMgr.obj
 0001:00001794       ??_C@_15HJEBGHIE@?$AAU?$AAp?$AA?$AA@ 10002794     LayoutManager:LayMgr.obj
 0001:000017a0       ??_C@_1HI@HIFNONDF@?$AAK?$AAe?$AAy?$AAb?$AAo?$AAa?$AAr?$AAd?$AA?3?$AA?5?$AAK?$AAe?$AAy?$AAp?$AAr?$AAe?$AAs?$AAs?$AA?5?$AAi?$AAg?$AAn?$AAo?$AAr?$AAe?$AAd?$AA?5?$AAs?$AAi?$AAn?$AAc?$AAe@ 100027a0     LayoutManager:LayMgr.obj
 0001:00001818       ??_C@_1CK@KHMJPINM@?$AAK?$AAe?$AAy?$AAb?$AAd?$AAE?$AAv?$AAe?$AAn?$AAt?$AAT?$AAh?$AAr?$AAe?$AAa?$AAd?$AAP?$AAr?$AAo?$AAc?$AA?$AA@ 10002818     LayoutManager:LayMgr.obj
 0001:00001848       ??_C@_1GA@ICNGPECE@?$AA?$CF?$AAs?$AA?3?$AA?5?$AAV?$AAK?$AA?3?$AA?5?$AA0?$AAx?$AA?$CF?$AA0?$AA8?$AAx?$AA?5?$AAS?$AAC?$AA?3?$AA?5?$AA0?$AAx?$AA?$CF?$AA0?$AA8?$AAx?$AA?5?$AAS?$AAh?$AAi?$AAf?$AAt?$AA?5@ 10002848     LayoutManager:LayMgr.obj
 0001:000018a8       ??_C@_1HA@NLAOBOAF@?$AAK?$AAe?$AAy?$AAb?$AAo?$AAa?$AAr?$AAd?$AA?3?$AA?5?$AAR?$AAe?$AAm?$AAa?$AAp?$AAp?$AAi?$AAn?$AAg?$AA?5?$AAf?$AAu?$AAn?$AAc?$AAt?$AAi?$AAo?$AAn?$AA?5?$AAr?$AAe?$AAt@ 100028a8     LayoutManager:LayMgr.obj
 0001:00001918       ??_C@_1CE@CMMKBGEA@?$AAS?$AAe?$AAn?$AAd?$AAR?$AAe?$AAm?$AAa?$AAp?$AAp?$AAe?$AAd?$AAE?$AAv?$AAe?$AAn?$AAt?$AA?$AA@ 10002918     LayoutManager:LayMgr.obj
 0001:00001940       ??_C@_1HE@LCAGGIGJ@?$AAK?$AAe?$AAy?$AAb?$AAo?$AAa?$AAr?$AAd?$AA?3?$AA?5?$AAE?$AAx?$AAc?$AAe?$AAp?$AAt?$AAi?$AAo?$AAn?$AA?5?$AAi?$AAn?$AA?5?$AAd?$AAe?$AAv?$AAi?$AAc?$AAe?$AA?5?$AAl?$AAa@ 10002940     LayoutManager:LayMgr.obj
 0001:000019b4       ??_C@_1CK@EJMAOEFN@?$AA?$CF?$AAs?$AA?3?$AA?5?$AAE?$AAx?$AAi?$AAt?$AAi?$AAn?$AAg?$AA?5?$AAt?$AAh?$AAr?$AAe?$AAa?$AAd?$AA?$AN?$AA?6?$AA?$AA@ 100029b4     LayoutManager:LayMgr.obj
 0001:000019e0       ??_C@_1GM@GEJDKGOI@?$AA?$CF?$AAs?$AA?3?$AA?5?$AAI?$AAO?$AAC?$AAT?$AAL?$AA_?$AAK?$AAB?$AAD?$AA_?$AAS?$AAE?$AAT?$AA_?$AAL?$AAO?$AAC?$AAA?$AAL?$AAE?$AA_?$AAF?$AAL?$AAA?$AAG?$AAS?$AA?5?$AAf@ 100029e0     LayoutManager:LayMgr.obj
 0001:00001a50       ??_C@_1GI@MGIEJLGL@?$AA?$CF?$AAs?$AA?3?$AA?5?$AAI?$AAO?$AAC?$AAT?$AAL?$AA_?$AAK?$AAB?$AAD?$AA_?$AAS?$AAE?$AAT?$AA_?$AAA?$AAU?$AAT?$AAO?$AAR?$AAE?$AAP?$AAE?$AAA?$AAT?$AA?5?$AAf?$AAa?$AAi@ 10002a50     LayoutManager:LayMgr.obj
 0001:00001ab8       ??_C@_1GG@OLCCOCA@?$AA?$CF?$AAs?$AA?3?$AA?5?$AAI?$AAO?$AAC?$AAT?$AAL?$AA_?$AAK?$AAB?$AAD?$AA_?$AAS?$AAE?$AAT?$AA_?$AAM?$AAO?$AAD?$AAI?$AAF?$AAI?$AAE?$AAR?$AAS?$AA?5?$AAf?$AAa?$AAi?$AAl@ 10002ab8     LayoutManager:LayMgr.obj
 0001:00001b20       ??_C@_1FE@LFKMDCMD@?$AA?$CF?$AAs?$AA?3?$AA?5?$AAC?$AAo?$AAu?$AAl?$AAd?$AA?5?$AAn?$AAo?$AAt?$AA?5?$AAc?$AAr?$AAe?$AAa?$AAt?$AAe?$AA?5?$AAf?$AAi?$AAl?$AAe?$AA?5?$AAo?$AAn?$AA?5?$AA?$CF?$AAs?$AA?5@ 10002b20     LayoutManager:LayMgr.obj
 0001:00001b78       ??_C@_1FI@JGHPMHHM@?$AA?$CF?$AAs?$AA?3?$AA?5?$AAN?$AAo?$AAt?$AAi?$AAf?$AAi?$AAc?$AAa?$AAt?$AAi?$AAo?$AAn?$AA?5?$AAf?$AAr?$AAo?$AAm?$AA?5?$AAn?$AAo?$AAn?$AA?5?$AAK?$AAB?$AAD?$AA?5?$AAd?$AAe@ 10002b78     LayoutManager:LayMgr.obj
 0001:00001bd0       ??_C@_17LIMMJKCA@?$AAK?$AAB?$AAD?$AA?$AA@ 10002bd0     LayoutManager:LayMgr.obj
 0001:00001bd8       ??_C@_1DO@KMEKPCAJ@?$AA?$CF?$AAs?$AA?3?$AA?5?$AAR?$AAe?$AAc?$AAe?$AAi?$AAv?$AAe?$AAd?$AA?5?$AA?$CF?$AAs?$AA?5?$AAn?$AAo?$AAt?$AAi?$AAf?$AAi?$AAc?$AAa?$AAt?$AAi?$AAo?$AAn?$AA?$AN?$AA?6?$AA?$AA@ 10002bd8     LayoutManager:LayMgr.obj
 0001:00001c18       ??_C@_1EI@GJEDBFAJ@?$AA?$CF?$AAs?$AA?3?$AA?5?$AAR?$AAe?$AAa?$AAd?$AAM?$AAs?$AAg?$AAQ?$AAu?$AAe?$AAu?$AAe?$AA?5?$AAf?$AAa?$AAi?$AAl?$AAe?$AAd?$AA?0?$AA?5?$AAe?$AAr?$AAr?$AAo?$AAr?$AA?5?$AA?$CF@ 10002c18     LayoutManager:LayMgr.obj
 0001:00001c60       ??_C@_1GG@EJCOGMMI@?$AA?$CF?$AAs?$AA?3?$AA?5?$AAW?$AAa?$AAi?$AAt?$AAF?$AAo?$AAr?$AAM?$AAu?$AAl?$AAt?$AAi?$AAp?$AAl?$AAe?$AAO?$AAb?$AAj?$AAe?$AAc?$AAt?$AAs?$AA?5?$AAr?$AAe?$AAt?$AAu?$AAr@ 10002c60     LayoutManager:LayMgr.obj
 0001:00001cc8       ??_C@_1GK@DJDBDDMM@?$AA?$CF?$AAs?$AA?3?$AA?5?$AAU?$AAn?$AAa?$AAb?$AAl?$AAe?$AA?5?$AAt?$AAo?$AA?5?$AAR?$AAe?$AAq?$AAu?$AAe?$AAs?$AAt?$AAD?$AAe?$AAv?$AAi?$AAc?$AAe?$AAN?$AAo?$AAt?$AAi?$AAf@ 10002cc8     LayoutManager:LayMgr.obj
 0001:00001d38       ??_C@_1FO@JDBJHEHH@?$AA?$CF?$AAs?$AA?3?$AA?5?$AAU?$AAn?$AAa?$AAb?$AAl?$AAe?$AA?5?$AAt?$AAo?$AA?5?$AAc?$AAr?$AAe?$AAa?$AAt?$AAe?$AA?5?$AAm?$AAe?$AAs?$AAs?$AAa?$AAg?$AAe?$AA?5?$AAq?$AAu?$AAe@ 10002d38     LayoutManager:LayMgr.obj
 0001:00001d98       ??_C@_1CM@HCCHLAFC@?$AAK?$AAb?$AAd?$AAN?$AAo?$AAt?$AAi?$AAf?$AAi?$AAc?$AAa?$AAt?$AAi?$AAo?$AAn?$AAT?$AAh?$AAr?$AAe?$AAa?$AAd?$AA?$AA@ 10002d98     LayoutManager:LayMgr.obj
 0001:00001dc8       ??_C@_1MA@BJKCJGPL@?$AA?$CF?$AAs?$AA?3?$AA?5?$AAN?$AAo?$AA?5?$AAk?$AAe?$AAy?$AAb?$AAo?$AAa?$AAr?$AAd?$AA?5?$AAl?$AAa?$AAy?$AAo?$AAu?$AAt?$AA?5?$AAw?$AAa?$AAs?$AA?5?$AAf?$AAo?$AAu?$AAn?$AAd@ 10002dc8     LayoutManager:LayMgr.obj
 0001:00001e88       ??_C@_1EG@LKPPLLLP@?$AA?$CF?$AAs?$AA?3?$AA?5?$AAN?$AAo?$AA?5?$AAv?$AAa?$AAl?$AAi?$AAd?$AA?5?$AAu?$AAn?$AAn?$AAa?$AAm?$AAe?$AAd?$AA?5?$AAp?$AAr?$AAe?$AAl?$AAo?$AAa?$AAd?$AA?5?$AAk?$AAe?$AAy@ 10002e88     LayoutManager:LayMgr.obj
 0001:00001ed0       ??_C@_1DE@ECMOJBFK@?$AAG?$AAe?$AAt?$AAD?$AAe?$AAf?$AAa?$AAu?$AAl?$AAt?$AAI?$AAn?$AAp?$AAu?$AAt?$AAM?$AAe?$AAt?$AAh?$AAo?$AAd?$AAN?$AAa?$AAm?$AAe?$AA?$AA@ 10002ed0     LayoutManager:LayMgr.obj
 0001:00001f08       ??_C@_1EK@OEKFGJMH@?$AA?$CF?$AAs?$AA?3?$AA?5?$AAP?$AAr?$AAe?$AAl?$AAo?$AAa?$AAd?$AA?5?$AAk?$AAe?$AAy?$AA?5?$AA?$CF?$AAu?$AA?5?$AAh?$AAa?$AAs?$AA?5?$AAa?$AA?5?$AAb?$AAa?$AAd?$AA?5?$AAv?$AAa?$AAl@ 10002f08     LayoutManager:LayMgr.obj
 0001:00001f54       ??_C@_1DE@OJAEHHEL@?$AAG?$AAe?$AAt?$AAP?$AAr?$AAe?$AAl?$AAo?$AAa?$AAd?$AAI?$AAn?$AAp?$AAu?$AAt?$AAM?$AAe?$AAt?$AAh?$AAo?$AAd?$AAN?$AAa?$AAm?$AAe?$AA?$AA@ 10002f54     LayoutManager:LayMgr.obj
 0001:00001f88       ??_C@_15EFLNJKHH@?$AA?$CF?$AAu?$AA?$AA@ 10002f88     LayoutManager:LayMgr.obj
 0001:00001f90       ??_C@_1FE@FBMCGJLE@?$AA?$CF?$AAs?$AA?3?$AA?5?$AAC?$AAo?$AAu?$AAl?$AAd?$AA?5?$AAn?$AAo?$AAt?$AA?5?$AAo?$AAp?$AAe?$AAn?$AA?5?$AAP?$AAr?$AAe?$AAl?$AAo?$AAa?$AAd?$AA?5?$AAr?$AAe?$AAg?$AAi?$AAs@ 10002f90     LayoutManager:LayMgr.obj
 0001:00001fe4       ??_C@_1DC@BLLENJMD@?$AAG?$AAe?$AAt?$AAP?$AAr?$AAe?$AAl?$AAo?$AAa?$AAd?$AAI?$AAn?$AAp?$AAu?$AAt?$AAM?$AAe?$AAt?$AAh?$AAo?$AAd?$AAK?$AAe?$AAy?$AA?$AA@ 10002fe4     LayoutManager:LayMgr.obj
 0001:0000201c       ??_C@_1DA@FKJDDCGN@?$AAK?$AAe?$AAy?$AAb?$AAo?$AAa?$AAr?$AAd?$AA?5?$AAL?$AAa?$AAy?$AAo?$AAu?$AAt?$AA?2?$AAP?$AAr?$AAe?$AAl?$AAo?$AAa?$AAd?$AA?$AA@ 1000301c     LayoutManager:LayMgr.obj
 0001:00002050       ??_C@_1EI@KLDFCHDI@?$AA?$CF?$AAs?$AA?3?$AA?5?$AAU?$AAn?$AAn?$AAa?$AAm?$AAe?$AAd?$AA?5?$AAP?$AAr?$AAe?$AAl?$AAo?$AAa?$AAd?$AA?5?$AAv?$AAa?$AAl?$AAu?$AAe?$AA?5?$AAi?$AAs?$AA?5?$AAb?$AAa?$AAd@ 10003050     LayoutManager:LayMgr.obj
 0001:00002098       ??_C@_1CO@FEKOBNID@?$AAG?$AAe?$AAt?$AAP?$AAr?$AAe?$AAl?$AAo?$AAa?$AAd?$AAU?$AAn?$AAN?$AAa?$AAm?$AAe?$AAd?$AAV?$AAa?$AAl?$AAu?$AAe?$AA?$AA@ 10003098     LayoutManager:LayMgr.obj
 0001:000020c8       ??_C@_1FI@IHOACNGN@?$AAI?$AAn?$AAv?$AAa?$AAl?$AAi?$AAd?$AA?5?$AAi?$AAn?$AAp?$AAu?$AAt?$AA?5?$AAl?$AAa?$AAn?$AAg?$AAu?$AAa?$AAg?$AAe?$AA?5?$AAi?$AAn?$AAf?$AAo?$AAr?$AAm?$AAa?$AAt?$AAi@ 100030c8     LayoutManager:LayMgr.obj
 0001:00002120       ??_C@_1FM@PFEDIBOM@?$AA?$CF?$AAs?$AA?3?$AA?5?$AAI?$AAn?$AAp?$AAu?$AAt?$AA?5?$AAl?$AAa?$AAn?$AAg?$AAu?$AAa?$AAg?$AAe?$AA?5?$AAe?$AAn?$AAt?$AAr?$AAy?$AA?5?$AAf?$AAu?$AAn?$AAc?$AAt?$AAi?$AAo@ 10003120     LayoutManager:LayMgr.obj
 0001:00002180       ??_C@_1EK@CFGLEGKN@?$AA?$CF?$AAs?$AA?3?$AA?5?$AAE?$AAx?$AAc?$AAe?$AAp?$AAt?$AAi?$AAo?$AAn?$AA?5?$AAi?$AAn?$AA?5?$AAe?$AAn?$AAt?$AAr?$AAy?$AA?5?$AAf?$AAu?$AAn?$AAc?$AAt?$AAi?$AAo?$AAn?$AA?5@ 10003180     LayoutManager:LayMgr.obj
 0001:000021d0       ??_C@_1FM@KEHGOGLJ@?$AA?$CF?$AAs?$AA?3?$AA?5?$AAC?$AAo?$AAu?$AAl?$AAd?$AA?5?$AAn?$AAo?$AAt?$AA?5?$AAg?$AAe?$AAt?$AA?5?$AAt?$AAh?$AAe?$AA?5?$AAa?$AAd?$AAd?$AAr?$AAe?$AAs?$AAs?$AA?5?$AAo?$AAf@ 100031d0     LayoutManager:LayMgr.obj
 0001:00002230       ??_C@_1GA@NGOLJMCD@?$AA?$CF?$AAs?$AA?3?$AA?5?$AAF?$AAa?$AAi?$AAl?$AAe?$AAd?$AA?5?$AAl?$AAo?$AAa?$AAd?$AAi?$AAn?$AAg?$AA?5?$AA?$CF?$AAs?$AA?5?$AAf?$AAo?$AAr?$AA?5?$AAi?$AAn?$AAp?$AAu?$AAt?$AA?5@ 10003230     LayoutManager:LayMgr.obj
 0001:00002290       ??_C@_1FI@BOEFILPH@?$AA?$CF?$AAs?$AA?3?$AA?5?$AAC?$AAo?$AAu?$AAl?$AAd?$AA?5?$AAn?$AAo?$AAt?$AA?5?$AAc?$AAh?$AAa?$AAn?$AAg?$AAe?$AA?5?$AAt?$AAo?$AA?5?$AAi?$AAn?$AAp?$AAu?$AAt?$AA?5?$AAl?$AAa@ 10003290     LayoutManager:LayMgr.obj
 0001:000022e8       ??_C@_1GI@LFCDMIGI@?$AA?$CF?$AAs?$AA?3?$AA?5?$AAC?$AAh?$AAa?$AAn?$AAg?$AAi?$AAn?$AAg?$AA?5?$AAf?$AAr?$AAo?$AAm?$AA?5?$AAi?$AAn?$AAp?$AAu?$AAt?$AA?5?$AAl?$AAa?$AAn?$AAg?$AAu?$AAa?$AAg?$AAe@ 100032e8     LayoutManager:LayMgr.obj
 0001:00002350       ??_C@_1CC@COBCHGHN@?$AAS?$AAe?$AAt?$AAI?$AAn?$AAp?$AAu?$AAt?$AAL?$AAa?$AAn?$AAg?$AAu?$AAa?$AAg?$AAe?$AA?$AA@ 10003350     LayoutManager:LayMgr.obj
 0001:00002374       ??_C@_19NGFMKOON@?$AA?$CF?$AA0?$AA8?$AAX?$AA?$AA@ 10003374     LayoutManager:LayMgr.obj
 0001:00002380       ??_C@_1DK@LEHEMEEF@?$AA?$CF?$AAs?$AA?3?$AA?5?$AAP?$AAr?$AAo?$AAb?$AAl?$AAe?$AAm?$AA?5?$AAr?$AAe?$AAa?$AAd?$AAi?$AAn?$AAg?$AA?5?$AAk?$AAe?$AAy?$AA?5?$AA?$CF?$AAs?$AA?$AN?$AA?6?$AA?$AA@ 10003380     LayoutManager:LayMgr.obj
 0001:000023c0       ??_C@_1EO@DNIHBIEC@?$AA?$CF?$AAs?$AA?3?$AA?5?$AAC?$AAo?$AAu?$AAl?$AAd?$AA?5?$AAn?$AAo?$AAt?$AA?5?$AAo?$AAp?$AAe?$AAn?$AA?5?$AAk?$AAe?$AAy?$AA?5?$AAf?$AAo?$AAr?$AA?5?$AAl?$AAa?$AAy?$AAo?$AAu@ 100033c0     LayoutManager:LayMgr.obj
 0001:00002410       ??_C@_1DI@DHJFPFMB@?$AA?$CF?$AAs?$AA?3?$AA?5?$AAC?$AAo?$AAu?$AAl?$AAd?$AA?5?$AAn?$AAo?$AAt?$AA?5?$AAo?$AAp?$AAe?$AAn?$AA?5?$AA?$CF?$AAs?$AA?5?$AAk?$AAe?$AAy?$AA?$AN?$AA?6?$AA?$AA@ 10003410     LayoutManager:LayMgr.obj
 0001:00002448       ??_C@_1CG@PFDANLGN@?$AAG?$AAe?$AAt?$AAI?$AAn?$AAp?$AAu?$AAt?$AAM?$AAe?$AAt?$AAh?$AAo?$AAd?$AAI?$AAn?$AAf?$AAo?$AA?$AA@ 10003448     LayoutManager:LayMgr.obj
 0001:00002470       ??_C@_1EI@CBNEBNIN@?$AA?$CF?$AAs?$AA?3?$AA?5?$AAN?$AAo?$AA?5?$AAm?$AAo?$AAd?$AAi?$AAf?$AAi?$AAe?$AAr?$AA?5?$AAm?$AAa?$AAt?$AAc?$AAh?$AA?5?$AAf?$AAo?$AAr?$AA?5?$AAv?$AAk?$AAe?$AAy?$AA?5?$AA?$CF@ 10003470     LayoutManager:LayMgr.obj
 0001:000024b8       ??_C@_1FA@GPKCAJJF@?$AA?$CF?$AAs?$AA?3?$AA?5?$AAE?$AAx?$AAc?$AAe?$AAe?$AAd?$AAe?$AAd?$AA?5?$AAm?$AAa?$AAx?$AA?5?$AAm?$AAo?$AAd?$AAi?$AAf?$AAi?$AAe?$AAr?$AA?5?$AAc?$AAo?$AAu?$AAn?$AAt?$AA?5@ 100034b8     LayoutManager:LayMgr.obj
 0001:00002508       ??_C@_1DK@OIFLDFBG@?$AAG?$AAe?$AAn?$AAe?$AAr?$AAa?$AAt?$AAe?$AAM?$AAo?$AAd?$AAi?$AAf?$AAi?$AAe?$AAr?$AAT?$AAo?$AAS?$AAh?$AAi?$AAf?$AAt?$AAT?$AAa?$AAb?$AAl?$AAe?$AA?$AA@ 10003508     LayoutManager:LayMgr.obj
 0001:00002548       ??_C@_1FC@JLOKMJPH@?$AA?$CF?$AAs?$AA?3?$AA?5?$AAC?$AAo?$AAu?$AAl?$AAd?$AA?5?$AAn?$AAo?$AAt?$AA?5?$AAr?$AAe?$AAa?$AAd?$AA?5?$AAv?$AAa?$AAl?$AAu?$AAe?$AA?5?$AAo?$AAf?$AA?5?$AA?$CF?$AAs?$AA?2?$AA?$CF@ 10003548     LayoutManager:LayMgr.obj
 0001:000025a0       ??_C@_1DO@PFNKHIDG@?$AA?$CF?$AAs?$AA?3?$AA?5?$AAC?$AAo?$AAu?$AAl?$AAd?$AA?5?$AAn?$AAo?$AAt?$AA?5?$AAo?$AAp?$AAe?$AAn?$AA?5?$AA?$CF?$AAs?$AA?2?$AA?$CF?$AAs?$AA?5?$AAk?$AAe?$AAy?$AA?$AN?$AA?6?$AA?$AA@ 100035a0     LayoutManager:LayMgr.obj
 0001:000025e0       ??_C@_1CK@DNDHAOAA@?$AAG?$AAe?$AAt?$AAI?$AAm?$AAe?$AAK?$AAe?$AAy?$AAb?$AAo?$AAa?$AAr?$AAd?$AAL?$AAa?$AAy?$AAo?$AAu?$AAt?$AA?$AA@ 100035e0     LayoutManager:LayMgr.obj
 0001:0000260c       ??_C@_1CA@GLIJBCFK@?$AAK?$AAe?$AAy?$AAb?$AAo?$AAa?$AAr?$AAd?$AA?5?$AAL?$AAa?$AAy?$AAo?$AAu?$AAt?$AA?$AA@ 1000360c     LayoutManager:LayMgr.obj
 0001:00002630       ??_C@_1EC@HAGJGNMN@?$AA?$CF?$AAs?$AA?3?$AA?5?$AAP?$AAr?$AAo?$AAc?$AA?5?$AAn?$AAa?$AAm?$AAe?$AA?5?$AA?$CC?$AA?$CF?$AAs?$AA?$CC?$AA?5?$AAi?$AAs?$AA?5?$AAt?$AAo?$AAo?$AA?5?$AAl?$AAo?$AAn?$AAg?$AA?$AN?$AA?6@ 10003630     LayoutManager:LayMgr.obj
 0001:00002674       ??_C@_1CI@LMGBELGL@?$AAG?$AAe?$AAt?$AAK?$AAe?$AAy?$AAb?$AAo?$AAa?$AAr?$AAd?$AAP?$AAr?$AAo?$AAc?$AAA?$AAd?$AAd?$AAr?$AA?$AA@ 10003674     LayoutManager:LayMgr.obj
 0001:000026a0       ??_C@_1FG@IKEAAOND@?$AAI?$AAn?$AAv?$AAa?$AAl?$AAi?$AAd?$AA?5?$AAd?$AAe?$AAv?$AAi?$AAc?$AAe?$AA?5?$AAl?$AAa?$AAy?$AAo?$AAu?$AAt?$AA?5?$AAi?$AAn?$AAf?$AAo?$AAr?$AAm?$AAa?$AAt?$AAi?$AAo@ 100036a0     LayoutManager:LayMgr.obj
 0001:000026f8       ??_C@_1FE@GONJHPLI@?$AA?$CF?$AAs?$AA?3?$AA?5?$AAD?$AAe?$AAv?$AAi?$AAc?$AAe?$AA?5?$AAl?$AAa?$AAy?$AAo?$AAu?$AAt?$AA?5?$AAe?$AAn?$AAt?$AAr?$AAy?$AA?5?$AAf?$AAu?$AAn?$AAc?$AAt?$AAi?$AAo?$AAn@ 100036f8     LayoutManager:LayMgr.obj
 0001:00002750       ??_C@_1FM@PGJBOEON@?$AA?$CF?$AAs?$AA?3?$AA?5?$AAU?$AAn?$AAa?$AAb?$AAl?$AAe?$AA?5?$AAt?$AAo?$AA?5?$AAl?$AAo?$AAa?$AAd?$AA?5?$AAd?$AAe?$AAv?$AAi?$AAc?$AAe?$AA?5?$AAl?$AAa?$AAy?$AAo?$AAu?$AAt@ 10003750     LayoutManager:LayMgr.obj
 0001:000027b0       ??_C@_1HO@LMMPANNC@?$AA?$CF?$AAs?$AA?3?$AA?5?$AAC?$AAo?$AAu?$AAl?$AAd?$AA?5?$AAn?$AAo?$AAt?$AA?5?$AAf?$AAi?$AAn?$AAd?$AA?5?$AAm?$AAa?$AAt?$AAc?$AAh?$AA?5?$AAP?$AAD?$AAD?$AA?5?$AA?$CF?$AAu?$AA?5@ 100037b0     LayoutManager:LayMgr.obj
 0001:00002830       ??_C@_1CA@IPKHFBAD@?$AAS?$AAe?$AAt?$AAD?$AAe?$AAv?$AAi?$AAc?$AAe?$AAL?$AAa?$AAy?$AAo?$AAu?$AAt?$AA?$AA@ 10003830     LayoutManager:LayMgr.obj
 0001:00002850       ??_C@_1FE@GAKCPDEP@?$AA?$CF?$AAs?$AA?3?$AA?5?$AAF?$AAa?$AAi?$AAl?$AAe?$AAd?$AA?5?$AAl?$AAo?$AAa?$AAd?$AAi?$AAn?$AAg?$AA?5?$AAd?$AAe?$AAv?$AAi?$AAc?$AAe?$AA?5?$AAl?$AAa?$AAy?$AAo?$AAu?$AAt@ 10003850     LayoutManager:LayMgr.obj
 0001:000028a4       ??_C@_1CK@LFKCMCDI@?$AAG?$AAe?$AAt?$AAD?$AAe?$AAv?$AAi?$AAc?$AAe?$AAL?$AAa?$AAy?$AAo?$AAu?$AAt?$AAE?$AAn?$AAt?$AAr?$AAy?$AA?$AA@ 100038a4     LayoutManager:LayMgr.obj
 0001:000028d0       ??_C@_1HC@KKNGAHGA@?$AA?$CF?$AAs?$AA?3?$AA?5?$AAF?$AAo?$AAu?$AAn?$AAd?$AA?5?$AAd?$AAe?$AAv?$AAi?$AAc?$AAe?$AA?5?$AAl?$AAa?$AAy?$AAo?$AAu?$AAt?$AA?5?$AAm?$AAa?$AAt?$AAc?$AAh?$AA?5?$AAf?$AAo@ 100038d0     LayoutManager:LayMgr.obj
 0001:00002948       ??_C@_1HG@CODMDNMO@?$AA?$CF?$AAs?$AA?3?$AA?5?$AAC?$AAo?$AAu?$AAl?$AAd?$AA?5?$AAn?$AAo?$AAt?$AA?5?$AAf?$AAi?$AAn?$AAd?$AA?5?$AAa?$AA?5?$AAd?$AAe?$AAv?$AAi?$AAc?$AAe?$AA?5?$AAl?$AAa?$AAy?$AAo@ 10003948     LayoutManager:LayMgr.obj
 0001:000029c0       ??_C@_1FG@HNPBMFMF@?$AA?$CF?$AAs?$AA?3?$AA?5?$AAN?$AAo?$AA?5?$AAd?$AAe?$AAv?$AAi?$AAc?$AAe?$AA?5?$AAl?$AAa?$AAy?$AAo?$AAu?$AAt?$AA?5?$AAs?$AAu?$AAb?$AAk?$AAe?$AAy?$AA?5?$AAf?$AAo?$AAu?$AAn@ 100039c0     LayoutManager:LayMgr.obj
 0001:00002a18       ??_C@_1CG@JNFKBALO@?$AAS?$AAe?$AAl?$AAe?$AAc?$AAt?$AAD?$AAe?$AAv?$AAi?$AAc?$AAe?$AAL?$AAa?$AAy?$AAo?$AAu?$AAt?$AA?$AA@ 10003a18     LayoutManager:LayMgr.obj
 0001:00002a40       ??_C@_1FO@GBIOBLJG@?$AA?$CF?$AAs?$AA?3?$AA?5?$AAE?$AAr?$AAr?$AAo?$AAr?$AA?5?$AAi?$AAn?$AA?5?$AAd?$AAe?$AAv?$AAi?$AAc?$AAe?$AA?5?$AAl?$AAa?$AAy?$AAo?$AAu?$AAt?$AA?5?$AAe?$AAn?$AAt?$AAr?$AAy@ 10003a40     LayoutManager:LayMgr.obj
 0001:00002aa0       ??_C@_1CO@OIGNLNDP@?$AAD?$AAe?$AAv?$AAi?$AAc?$AAe?$AAL?$AAa?$AAy?$AAo?$AAu?$AAt?$AAM?$AAa?$AAt?$AAc?$AAh?$AAe?$AAs?$AAP?$AAD?$AAD?$AA?$AA@ 10003aa0     LayoutManager:LayMgr.obj
 0001:00002ad0       ??_C@_1M@LLCLNBHO@?$AA?$CF?$AAs?$AA_?$AA?$CF?$AAs?$AA?$AA@ 10003ad0     LayoutManager:LayMgr.obj
 0001:00002adc       ??_C@_1M@FKDMEONL@?$AA?9?$AA?$CF?$AAs?$AA?$AN?$AA?6?$AA?$AA@ 10003adc     LayoutManager:LayMgr.obj
 0001:00002ae8       ??_C@_1M@LFABOLDL@?$AA?$CL?$AA?$CF?$AAs?$AA?$AN?$AA?6?$AA?$AA@ 10003ae8     LayoutManager:LayMgr.obj
 0001:00002af4       ??_C@_1DC@IFJFLG@?$AAL?$AAa?$AAy?$AAo?$AAu?$AAt?$AAM?$AAg?$AAr?$AAG?$AAe?$AAt?$AAK?$AAe?$AAy?$AAb?$AAo?$AAa?$AAr?$AAd?$AAT?$AAy?$AAp?$AAe?$AA?$AA@ 10003af4     LayoutManager:LayMgr.obj
 0001:00002b28       ??_C@_1FA@KNOLPHGM@?$AA?$CF?$AAs?$AA?3?$AA?5?$AAM?$AAu?$AAs?$AAt?$AA?5?$AAb?$AAe?$AA?5?$AAc?$AAa?$AAl?$AAl?$AAe?$AAd?$AA?5?$AAw?$AAi?$AAt?$AAh?$AA?5?$AAi?$AAd?$AAT?$AAh?$AAr?$AAe?$AAa?$AAd@ 10003b28     LayoutManager:LayMgr.obj
 0001:00002b78       ??_C@_1DG@IKNCCLA@?$AAL?$AAa?$AAy?$AAo?$AAu?$AAt?$AAM?$AAg?$AAr?$AAG?$AAe?$AAt?$AAK?$AAe?$AAy?$AAb?$AAo?$AAa?$AAr?$AAd?$AAL?$AAa?$AAy?$AAo?$AAu?$AAt?$AA?$AA@ 10003b78     LayoutManager:LayMgr.obj
 0001:00002bb0       ??_C@_1DO@DPIGDLGA@?$AAL?$AAa?$AAy?$AAo?$AAu?$AAt?$AAM?$AAg?$AAr?$AAG?$AAe?$AAt?$AAK?$AAe?$AAy?$AAb?$AAo?$AAa?$AAr?$AAd?$AAL?$AAa?$AAy?$AAo?$AAu?$AAt?$AAN?$AAa?$AAm?$AAe?$AA?$AA@ 10003bb0     LayoutManager:LayMgr.obj
 0001:00002bf0       ??_C@_1EM@DEAGOFCP@?$AA?$CF?$AAs?$AA?3?$AA?5?$AAB?$AAu?$AAf?$AAf?$AAe?$AAr?$AA?5?$AAs?$AAi?$AAz?$AAe?$AA?5?$AAi?$AAs?$AA?5?$AAn?$AAo?$AAt?$AA?5?$AAl?$AAa?$AAr?$AAg?$AAe?$AA?5?$AAe?$AAn?$AAo@ 10003bf0     LayoutManager:LayMgr.obj
 0001:00002c3c       ??_C@_1DO@DJOPKDPJ@?$AAL?$AAa?$AAy?$AAo?$AAu?$AAt?$AAM?$AAg?$AAr?$AAG?$AAe?$AAt?$AAK?$AAe?$AAy?$AAb?$AAo?$AAa?$AAr?$AAd?$AAL?$AAa?$AAy?$AAo?$AAu?$AAt?$AAL?$AAi?$AAs?$AAt?$AA?$AA@ 10003c3c     LayoutManager:LayMgr.obj
 0001:00002c80       ??_C@_1GO@LPEEAFIF@?$AA?$CF?$AAs?$AA?3?$AA?5?$AAS?$AAu?$AAc?$AAc?$AAe?$AAs?$AAs?$AAf?$AAu?$AAl?$AAl?$AAy?$AA?5?$AAl?$AAo?$AAa?$AAd?$AAe?$AAd?$AA?5?$AAl?$AAa?$AAy?$AAo?$AAu?$AAt?$AA?5?$AA?$CF@ 10003c80     LayoutManager:LayMgr.obj
 0001:00002cf0       ??_C@_1GE@FCKLEHDD@?$AA?$CF?$AAs?$AA?3?$AA?5?$AAC?$AAo?$AAu?$AAl?$AAd?$AA?5?$AAn?$AAo?$AAt?$AA?5?$AAs?$AAe?$AAt?$AA?5?$AAd?$AAe?$AAf?$AAa?$AAu?$AAl?$AAt?$AA?5?$AAv?$AAa?$AAl?$AAu?$AAe?$AA?5@ 10003cf0     LayoutManager:LayMgr.obj
 0001:00002d58       ??_C@_1EM@MEIACPAD@?$AA?$CF?$AAs?$AA?3?$AA?5?$AAC?$AAo?$AAu?$AAl?$AAd?$AA?5?$AAn?$AAo?$AAt?$AA?5?$AAc?$AAr?$AAe?$AAa?$AAt?$AAe?$AA?5?$AAp?$AAr?$AAe?$AAl?$AAo?$AAa?$AAd?$AA?5?$AAk?$AAe?$AAy@ 10003d58     LayoutManager:LayMgr.obj
 0001:00002da8       ??_C@_1EC@OHHNMJOD@?$AA?$CF?$AAs?$AA?3?$AA?5?$AAC?$AAo?$AAu?$AAl?$AAd?$AA?5?$AAn?$AAo?$AAt?$AA?5?$AAo?$AAp?$AAe?$AAn?$AA?5?$AAp?$AAr?$AAe?$AAl?$AAo?$AAa?$AAd?$AA?5?$AAk?$AAe?$AAy?$AA?$AN?$AA?6@ 10003da8     LayoutManager:LayMgr.obj
 0001:00002df0       ??_C@_1GA@BALBINBG@?$AA?$CF?$AAs?$AA?3?$AA?5?$AAC?$AAo?$AAu?$AAl?$AAd?$AA?5?$AAn?$AAo?$AAt?$AA?5?$AAf?$AAi?$AAn?$AAd?$AA?5?$AAa?$AAn?$AA?5?$AAa?$AAv?$AAa?$AAi?$AAl?$AAa?$AAb?$AAl?$AAe?$AA?5@ 10003df0     LayoutManager:LayMgr.obj
 0001:00002e50       ??_C@_1EE@JFJJNEJC@?$AA?$CF?$AAs?$AA?3?$AA?5?$AAL?$AAa?$AAy?$AAo?$AAu?$AAt?$AA?5?$AA?$CF?$AAs?$AA?5?$AAi?$AAs?$AA?5?$AAa?$AAl?$AAr?$AAe?$AAa?$AAd?$AAy?$AA?5?$AAl?$AAo?$AAa?$AAd?$AAe?$AAd?$AA?$AN@ 10003e50     LayoutManager:LayMgr.obj
 0001:00002e94       ??_C@_1CM@BKEFHEAE@?$AA?$CF?$AAs?$AA?3?$AA?5?$AAF?$AAo?$AAu?$AAn?$AAd?$AA?5?$AAl?$AAa?$AAy?$AAo?$AAu?$AAt?$AA?5?$AA?$CF?$AAs?$AA?$AN?$AA?6?$AA?$AA@ 10003e94     LayoutManager:LayMgr.obj
 0001:00002ec0       ??_C@_1FC@MCCKLOEL@?$AA?$CF?$AAs?$AA?3?$AA?5?$AAR?$AAe?$AAq?$AAu?$AAe?$AAs?$AAt?$AAe?$AAd?$AA?5?$AAl?$AAa?$AAy?$AAo?$AAu?$AAt?$AA?5?$AA?$CF?$AAs?$AA?5?$AAd?$AAo?$AAe?$AAs?$AA?5?$AAn?$AAo?$AAt@ 10003ec0     LayoutManager:LayMgr.obj
 0001:00002f18       ??_C@_1FA@KAMPNMAH@?$AA?$CF?$AAs?$AA?3?$AA?5?$AAK?$AAe?$AAy?$AAb?$AAo?$AAa?$AAr?$AAd?$AA?5?$AAl?$AAa?$AAy?$AAo?$AAu?$AAt?$AA?5?$AA?$CF?$AAs?$AA?5?$AAd?$AAo?$AAe?$AAs?$AA?5?$AAn?$AAo?$AAt?$AA?5@ 10003f18     LayoutManager:LayMgr.obj
 0001:00002f68       ??_C@_1DE@OEKJAIHK@?$AA?$CF?$AAs?$AA?3?$AA?5?$AA?$CF?$AAs?$AA?5?$AAi?$AAs?$AA?5?$AAa?$AAn?$AA?5?$AAi?$AAn?$AAv?$AAa?$AAl?$AAi?$AAd?$AA?5?$AAi?$AAd?$AA?$AN?$AA?6?$AA?$AA@ 10003f68     LayoutManager:LayMgr.obj
 0001:00002f9c       ??_C@_1DI@JHLFHMPL@?$AAL?$AAa?$AAy?$AAo?$AAu?$AAt?$AAM?$AAg?$AAr?$AAL?$AAo?$AAa?$AAd?$AAK?$AAe?$AAy?$AAb?$AAo?$AAa?$AAr?$AAd?$AAL?$AAa?$AAy?$AAo?$AAu?$AAt?$AA?$AA@ 10003f9c     LayoutManager:LayMgr.obj
 0001:00002fd8       ??_C@_1LO@CODLIIHA@?$AA?$CF?$AAs?$AA?3?$AA?5?$AAF?$AAa?$AAi?$AAl?$AAu?$AAr?$AAe?$AA?5?$AAs?$AAe?$AAt?$AAt?$AAi?$AAn?$AAg?$AA?5?$AAd?$AAe?$AAv?$AAi?$AAc?$AAe?$AA?5?$AAl?$AAa?$AAy?$AAo?$AAu@ 10003fd8     LayoutManager:LayMgr.obj
 0001:00003098       ??_C@_1KO@BLOFMLMO@?$AA?$CF?$AAs?$AA?3?$AA?5?$AAF?$AAa?$AAi?$AAl?$AAu?$AAr?$AAe?$AA?5?$AAs?$AAe?$AAt?$AAt?$AAi?$AAn?$AAg?$AA?5?$AAi?$AAn?$AAp?$AAu?$AAt?$AA?5?$AAl?$AAa?$AAn?$AAg?$AAu?$AAa@ 10004098     LayoutManager:LayMgr.obj
 0001:00003148       ??_C@_1DO@NIMCJCOO@?$AA?$CF?$AAs?$AA?3?$AA?5?$AAC?$AAa?$AAl?$AAl?$AAe?$AAd?$AA?5?$AAw?$AAi?$AAt?$AAh?$AA?5?$AAh?$AAk?$AAl?$AA?5?$AA?$DN?$AA?5?$AA0?$AAx?$AA?$CF?$AA0?$AA8?$AAx?$AA?$AN?$AA?6?$AA?$AA@ 10004148     LayoutManager:LayMgr.obj
 0001:00003188       ??_C@_1EA@FIGMDCGA@?$AAL?$AAa?$AAy?$AAo?$AAu?$AAt?$AAM?$AAg?$AAr?$AAA?$AAc?$AAt?$AAi?$AAv?$AAa?$AAt?$AAe?$AAK?$AAe?$AAy?$AAb?$AAo?$AAa?$AAr?$AAd?$AAL?$AAa?$AAy?$AAo?$AAu?$AAt?$AA?$AA@ 10004188     LayoutManager:LayMgr.obj
 0001:000031c8       ??_C@_1EM@JGHMPAIA@?$AAL?$AAa?$AAy?$AAo?$AAu?$AAt?$AA?5?$AAM?$AAa?$AAn?$AAa?$AAg?$AAe?$AAr?$AA?5?$AA?3?$AA?5?$AAD?$AAL?$AAL?$AA_?$AAP?$AAR?$AAO?$AAC?$AAE?$AAS?$AAS?$AA_?$AAA?$AAT?$AAT@ 100041c8     LayoutManager:LayMgr.obj
 0001:00003218       ??_C@_1EC@PDDNOLEO@?$AAK?$AAe?$AAr?$AAn?$AAe?$AAl?$AA?5?$AAP?$AAr?$AAo?$AAf?$AAi?$AAl?$AAe?$AAr?$AA?5?$AAm?$AAo?$AAd?$AAe?$AA?3?$AA?5?$AAB?$AAu?$AAf?$AAf?$AAe?$AAr?$AAe?$AAd?$AA?$AN?$AA?6@ 10004218     LayoutManager:profiler.obj
 0001:0000325c       ??_C@_1DM@LDFFLEGF@?$AAK?$AAe?$AAr?$AAn?$AAe?$AAl?$AA?5?$AAP?$AAr?$AAo?$AAf?$AAi?$AAl?$AAe?$AAr?$AA?5?$AAm?$AAo?$AAd?$AAe?$AA?3?$AA?5?$AAC?$AAe?$AAL?$AAo?$AAg?$AA?$AN?$AA?6?$AA?$AA@ 1000425c     LayoutManager:profiler.obj
 0001:00003298       ??_C@_1EG@OLMAKGJN@?$AAK?$AAe?$AAr?$AAn?$AAe?$AAl?$AA?5?$AAP?$AAr?$AAo?$AAf?$AAi?$AAl?$AAe?$AAr?$AA?5?$AAm?$AAo?$AAd?$AAe?$AA?3?$AA?5?$AAU?$AAn?$AAb?$AAu?$AAf?$AAf?$AAe?$AAr?$AAe?$AAd@ 10004298     LayoutManager:profiler.obj
 0001:000032e0       ??_C@_1BE@MPEJEKEH@?$AAK?$AAP?$AAP?$AAL?$AAa?$AAy?$AAo?$AAu?$AAt?$AA?$AA@ 100042e0     Keypad_mx25_topaz_v1:kbd.obj
 0001:000032f4       ??_C@_1DO@MEANBKIH@?$AAC?$AAo?$AAu?$AAl?$AAd?$AA?5?$AAn?$AAo?$AAt?$AA?5?$AAi?$AAn?$AAi?$AAt?$AAi?$AAa?$AAl?$AAi?$AAz?$AAe?$AA?5?$AAk?$AAe?$AAy?$AAp?$AAa?$AAd?$AA?4?$AA?$AN?$AA?6?$AA?$AA@ 100042f4     Keypad_mx25_topaz_v1:kbd.obj
 0001:00003338       ??_C@_1LK@KJIJBIHG@?$AAc?$AA?3?$AA?2?$AAw?$AAi?$AAn?$AAc?$AAe?$AAr?$AAo?$AAo?$AAt?$AAs?$AA?2?$AAt?$AAo?$AAp?$AAa?$AAz?$AA?2?$AAw?$AAi?$AAn?$AAc?$AAe?$AA7?$AA0?$AA0?$AA?2?$AAp?$AAl?$AAa@ 10004338     Keypad_mx25_topaz_v1:kbd.obj
 0001:000033f4       ??_C@_1DG@BACDDNAK@?$AA?$CF?$AAs?$AA?3?$AA?5?$AAI?$AAn?$AAi?$AAt?$AAi?$AAa?$AAl?$AAi?$AAz?$AAe?$AA?5?$AAK?$AAP?$AAP?$AA?5?$AAI?$AAD?$AA?5?$AA?$CF?$AAu?$AA?$AN?$AA?6?$AA?$AA@ 100043f4     Keypad_mx25_topaz_v1:kbd.obj
 0001:0000342c       ??_C@_1BE@MFGBOMPO@?$AAK?$AAP?$AAP?$AA_?$AAE?$AAn?$AAt?$AAr?$AAy?$AA?$AA@ 1000442c     Keypad_mx25_topaz_v1:kbd.obj
 0001:00003440       ??_C@_1CM@CNFNOMMH@?$AAK?$AAe?$AAy?$AAb?$AAd?$AAP?$AAd?$AAd?$AA_?$AAP?$AAo?$AAw?$AAe?$AAr?$AAH?$AAa?$AAn?$AAd?$AAl?$AAe?$AAr?$AA?$AA@ 10004440     Keypad_mx25_topaz_v1:keypad.obj
 0001:0000346c       ??_C@_1CC@NCEIAIOE@?$AAK?$AAp?$AAp?$AAI?$AAs?$AAr?$AAT?$AAh?$AAr?$AAe?$AAa?$AAd?$AAP?$AAr?$AAo?$AAc?$AA?$AA@ 1000446c     Keypad_mx25_topaz_v1:keypad.obj
 0001:00003490       ??_C@_1DG@MPBOBHG@?$AA?$CF?$AAs?$AA?3?$AA?5?$AAk?$AAe?$AAy?$AAp?$AAa?$AAd?$AA?5?$AAe?$AAv?$AAe?$AAn?$AAt?$AAs?$AA?5?$AA0?$AAx?$AA?$CF?$AA0?$AA8?$AAx?$AA?$AN?$AA?6?$AA?$AA@ 10004490     Keypad_mx25_topaz_v1:keypad.obj
 0001:000034c8       ??_C@_1FA@LIPICKON@?$AA?$CF?$AAs?$AA?3?$AA?5?$AAe?$AAv?$AAe?$AAn?$AAt?$AA?5?$AA0?$AAx?$AA?$CF?$AA0?$AA8?$AAx?$AA?3?$AA?5?$AAS?$AAc?$AAa?$AAn?$AAC?$AAo?$AAd?$AAe?$AA?5?$AA0?$AAx?$AA?$CF?$AA0?$AA8@ 100044c8     Keypad_mx25_topaz_v1:keypad.obj
 0001:00003518       ??_C@_1MA@GIFAAILO@?$AAc?$AA?3?$AA?2?$AAw?$AAi?$AAn?$AAc?$AAe?$AAr?$AAo?$AAo?$AAt?$AAs?$AA?2?$AAt?$AAo?$AAp?$AAa?$AAz?$AA?2?$AAw?$AAi?$AAn?$AAc?$AAe?$AA7?$AA0?$AA0?$AA?2?$AAp?$AAl?$AAa@ 10004518     Keypad_mx25_topaz_v1:keypad.obj
 0001:000035d8       ??_C@_1CK@CHLCGBHH@?$AAK?$AAe?$AAy?$AAb?$AAd?$AAP?$AAd?$AAd?$AA_?$AAG?$AAe?$AAt?$AAE?$AAv?$AAe?$AAn?$AAt?$AAE?$AAx?$AA2?$AA?$AA@ 100045d8     Keypad_mx25_topaz_v1:keypad.obj
 0001:00003608       ??_C@_1FC@JNHHONNA@?$AAK?$AAp?$AAp?$AAI?$AAs?$AAr?$AAT?$AAh?$AAr?$AAe?$AAa?$AAd?$AAS?$AAt?$AAa?$AAr?$AAt?$AA?3?$AA?5?$AAC?$AAr?$AAe?$AAa?$AAt?$AAe?$AAT?$AAh?$AAr?$AAe?$AAa?$AAd?$AA?5@ 10004608     Keypad_mx25_topaz_v1:keypad.obj
 0001:0000365c       ??_C@_1CE@HHBEDKOC@?$AAK?$AAp?$AAp?$AAI?$AAs?$AAr?$AAT?$AAh?$AAr?$AAe?$AAa?$AAd?$AAS?$AAt?$AAa?$AAr?$AAt?$AA?$AA@ 1000465c     Keypad_mx25_topaz_v1:keypad.obj
 0001:00003680       ??_C@_1EG@LGAKFIK@?$AA?$FL?$AAK?$AAP?$AAP?$AA?$FN?$AA?5?$AA?$CF?$AAs?$AA?3?$AA?5?$AAf?$AAa?$AAi?$AAl?$AA?5?$AAt?$AAo?$AA?5?$AAB?$AAS?$AAP?$AAK?$AAp?$AAp?$AAR?$AAe?$AAg?$AAI?$AAn?$AAi?$AAt?$AA?$CB@ 10004680     Keypad_mx25_topaz_v1:keypad.obj
 0001:000036c8       ??_C@_1EE@LJPNCNGB@?$AA?$FL?$AAK?$AAP?$AAP?$AA?$FN?$AA?$CF?$AAs?$AA?3?$AA?5?$AA?5?$AAi?$AAr?$AAq?$AA?$DN?$AA0?$AAx?$AA?$CF?$AAx?$AA?0?$AA?5?$AAs?$AAy?$AAs?$AAI?$AAr?$AAq?$AA?$DN?$AA0?$AAx?$AA?$CF?$AAx?$AA?$AN@ 100046c8     Keypad_mx25_topaz_v1:keypad.obj
 0001:00003710       ??_C@_1EI@MFIFPKAO@?$AA?$CF?$AAs?$AA?3?$AA?5?$AAD?$AAo?$AAn?$AAe?$AA?5?$AAe?$AAn?$AAa?$AAb?$AAl?$AAi?$AAn?$AAg?$AA?5?$AAt?$AAh?$AAe?$AA?5?$AAw?$AAa?$AAk?$AAe?$AA?5?$AAs?$AAo?$AAu?$AAr?$AAc@ 10004710     Keypad_mx25_topaz_v1:keypad.obj
 0001:00003758       ??_C@_1FI@DIHGJGMH@?$AA?$CF?$AAs?$AA?3?$AA?5?$AAA?$AAb?$AAo?$AAu?$AAt?$AA?5?$AAt?$AAo?$AA?5?$AAe?$AAn?$AAa?$AAb?$AAl?$AAe?$AA?5?$AAt?$AAh?$AAe?$AA?5?$AAw?$AAa?$AAk?$AAe?$AA?5?$AAs?$AAo?$AAu@ 10004758     Keypad_mx25_topaz_v1:keypad.obj
 0001:000037b0       ??_C@_1FK@POMEHCGJ@?$AAI?$AAs?$AAr?$AAT?$AAh?$AAr?$AAe?$AAa?$AAd?$AAP?$AAr?$AAo?$AAc?$AA?3?$AA?5?$AAK?$AAe?$AAy?$AAb?$AAd?$AAI?$AAn?$AAt?$AAe?$AAr?$AAr?$AAu?$AAp?$AAt?$AAE?$AAn?$AAa@ 100047b0     Keypad_mx25_topaz_v1:keypad.obj
 0001:00003810       ??_C@_1IA@JKNIKOOG@?$AAE?$AAR?$AAR?$AAO?$AAR?$AA?3?$AA?5?$AAF?$AAa?$AAi?$AAl?$AAe?$AAd?$AA?5?$AAt?$AAo?$AA?5?$AAo?$AAb?$AAt?$AAa?$AAi?$AAn?$AA?5?$AAs?$AAy?$AAs?$AAi?$AAn?$AAt?$AAr?$AA?5@ 10004810     Keypad_mx25_topaz_v1:keypad.obj
 0001:00003890       ??_C@_1EK@EALJNCCM@?$AAI?$AAs?$AAr?$AAT?$AAh?$AAr?$AAe?$AAa?$AAd?$AAP?$AAr?$AAo?$AAc?$AA?3?$AA?5?$AAI?$AAn?$AAt?$AAe?$AAr?$AAr?$AAu?$AAp?$AAt?$AAI?$AAn?$AAi?$AAt?$AAi?$AAa?$AAl?$AAi@ 10004890     Keypad_mx25_topaz_v1:keypad.obj
 0001:000038dc       ??_C@_1BM@COLJAECJ@?$AAK?$AAp?$AAp?$AAI?$AAn?$AAi?$AAt?$AAi?$AAa?$AAl?$AAi?$AAz?$AAe?$AA?$AA@ 100048dc     Keypad_mx25_topaz_v1:keypad.obj
 0001:000038f8       ??_C@_1GI@JEALIHMP@?$AAK?$AAe?$AAy?$AAb?$AAd?$AAI?$AAs?$AAt?$AAL?$AAo?$AAo?$AAp?$AA?3?$AA?5?$AAK?$AAe?$AAy?$AAb?$AAo?$AAa?$AAr?$AAd?$AA?5?$AAd?$AAr?$AAi?$AAv?$AAe?$AAr?$AA?5?$AAt?$AAh@ 100048f8     KeybdIst:KeybdIst.obj
 0001:00003960       ??_C@_1HO@FBEEIAMI@?$AAd?$AA?3?$AA?2?$AAc?$AAh?$AAe?$AAl?$AAa?$AAn?$AAr?$AAt?$AAm?$AA2?$AA?2?$AAp?$AAu?$AAb?$AAl?$AAi?$AAc?$AA?2?$AAc?$AAo?$AAm?$AAm?$AAo?$AAn?$AA?2?$AAo?$AAa?$AAk?$AA?2@ 10004960     KeybdIst:KeybdIst.obj
 0001:00003a04       KPPLayout                  10004a04 f   BSPKeypad:bspkeypad.obj
 0001:00003afc       ?BSPKppRegInit@@YAHXZ      10004afc f   BSPKeypad:bspkeypad.obj
 0001:00003fb8       ?BSPKPPGetScanCodes@@YAIQAIQAH@Z 10004fb8 f   BSPKeypad:bspkeypad.obj
 0001:00004ca8       ?BSPKppPowerOn@@YAHXZ      10005ca8 f   BSPKeypad:bspkeypad.obj
 0001:00004da8       ?BSPKppPowerOff@@YAHXZ     10005da8 f   BSPKeypad:bspkeypad.obj
 0001:00004edc       ?BSPKppSetClockGatingMode@@YAHH@Z 10005edc f   BSPKeypad:bspkeypad.obj
 0001:00004fcc       ?BSPKppIsWakeUpSource@@YAHXZ 10005fcc f   BSPKeypad:bspkeypad.obj
 0001:000051c4       IL_00000409                100061c4 f   InputLang_0409:IL_0409.obj
 0001:000052d0       ?TogglePDDLights@@YAXKI@Z  100062d0 f   LayoutManager:LayMgr.obj
 0001:00005498       ?ToggleLights@@YAXI@Z      10006498 f   LayoutManager:LayMgr.obj
 0001:000055dc       KeybdDriverVKeyToUnicode   100065dc f   LayoutManager:LayMgr.obj
 0001:00007f20       KeybdDriverInitStates      10008f20 f   LayoutManager:LayMgr.obj
 0001:00007f54       KeybdDriverMapVirtualKey   10008f54 f   LayoutManager:LayMgr.obj
 0001:000088e8       KeybdDriverGetInfo         100098e8 f   LayoutManager:LayMgr.obj
 0001:00008d3c       KeybdDriverSetMode         10009d3c f   LayoutManager:LayMgr.obj
 0001:00008f4c       KeybdDriverPowerHandler    10009f4c f   LayoutManager:LayMgr.obj
 0001:00009050       KeybdDriverSetPowerState   1000a050 f   LayoutManager:LayMgr.obj
 0001:000090d8       KeybdDriverGetPowerCaps    1000a0d8 f   LayoutManager:LayMgr.obj
 0001:00009184       KeybdDriverIOControl       1000a184 f   LayoutManager:LayMgr.obj
 0001:00009258       KeybdDriverDeinitializeEx  1000a258 f   LayoutManager:LayMgr.obj
 0001:00009514       KeybdDriverInitializeEx    1000a514 f   LayoutManager:LayMgr.obj
 0001:0000e770       LayoutMgrGetKeyboardType   1000f770 f   LayoutManager:LayMgr.obj
 0001:0000e890       LayoutMgrGetKeyboardLayout 1000f890 f   LayoutManager:LayMgr.obj
 0001:0000e998       LayoutMgrGetKeyboardLayoutName 1000f998 f   LayoutManager:LayMgr.obj
 0001:0000eafc       LayoutMgrGetKeyboardLayoutList 1000fafc f   LayoutManager:LayMgr.obj
 0001:0000ed64       LayoutMgrLoadKeyboardLayout 1000fd64 f   LayoutManager:LayMgr.obj
 0001:0000f5f0       LayoutMgrActivateKeyboardLayout 100105f0 f   LayoutManager:LayMgr.obj
 0001:0000f7d8       KeybdMDDRegisterCallbacks  100107d8 f   LayoutManager:LayMgr.obj
 0001:0000f8b4       KeybdMDDRegisterGUID       100108b4 f   LayoutManager:LayMgr.obj
 0001:0000f980       DllMain                    10010980 f   LayoutManager:LayMgr.obj
 0001:0000fa04       SetEvent                   10010a04 f i LayoutManager:LayMgr.obj
 0001:0000fa38       GetCurrentThread           10010a38 f i LayoutManager:LayMgr.obj
 0001:0000fa50       ?LAYOUT_HAS_KOREAN_KEYS@@YAHPAUHKL__@@@Z 10010a50 f i LayoutManager:LayMgr.obj
 0001:0000fab0       ?wcsstr@@YAPAGPAGPBG@Z     10010ab0 f i LayoutManager:LayMgr.obj
 0001:0000fae4       ?wcsrchr@@YAPAGPAGG@Z      10010ae4 f i LayoutManager:LayMgr.obj
 0001:0000fb18       ?DoProfilerKey@@YAHG@Z     10010b18 f   LayoutManager:profiler.obj
 0001:0000fc78       NKDbgPrintfW               10010c78 f   coredll:COREDLL.dll
 0001:0000fc88       Sleep                      10010c88 f   coredll:COREDLL.dll
 0001:0000fc98       LeaveCriticalSection       10010c98 f   coredll:COREDLL.dll
 0001:0000fca8       GetTickCount               10010ca8 f   coredll:COREDLL.dll
 0001:0000fcb8       EnterCriticalSection       10010cb8 f   coredll:COREDLL.dll
 0001:0000fcc8       InitializeCriticalSection  10010cc8 f   coredll:COREDLL.dll
 0001:0000fcd8       DeviceIoControl            10010cd8 f   coredll:COREDLL.dll
 0001:0000fce8       SetLastError               10010ce8 f   coredll:COREDLL.dll
 0001:0000fcf8       LocalFree                  10010cf8 f   coredll:COREDLL.dll
 0001:0000fd08       FreeLibrary                10010d08 f   coredll:COREDLL.dll
 0001:0000fd18       DeleteCriticalSection      10010d18 f   coredll:COREDLL.dll
 0001:0000fd28       CloseHandle                10010d28 f   coredll:COREDLL.dll
 0001:0000fd38       LocalAlloc                 10010d38 f   coredll:COREDLL.dll
 0001:0000fd48       CreateThread               10010d48 f   coredll:COREDLL.dll
 0001:0000fd58       CreateEventW               10010d58 f   coredll:COREDLL.dll
 0001:0000fd68       WaitForSingleObject        10010d68 f   coredll:COREDLL.dll
 0001:0000fd78       SetThreadPriority          10010d78 f   coredll:COREDLL.dll
 0001:0000fd88       EventModify                10010d88 f   coredll:COREDLL.dll
 0001:0000fd98       keybd_eventEx              10010d98 f   coredll:COREDLL.dll
 0001:0000fda8       WaitForMultipleObjects     10010da8 f   coredll:COREDLL.dll
 0001:0000fdb8       StopDeviceNotifications    10010db8 f   coredll:COREDLL.dll
 0001:0000fdc8       CreateFileW                10010dc8 f   coredll:COREDLL.dll
 0001:0000fdd8       ReadMsgQueue               10010dd8 f   coredll:COREDLL.dll
 0001:0000fde8       RequestDeviceNotifications 10010de8 f   coredll:COREDLL.dll
 0001:0000fdf8       GetLastError               10010df8 f   coredll:COREDLL.dll
 0001:0000fe08       CreateMsgQueue             10010e08 f   coredll:COREDLL.dll
 0001:0000fe18       StringCchCopyW             10010e18 f   coredll:COREDLL.dll
 0001:0000fe28       RegCloseKey                10010e28 f   coredll:COREDLL.dll
 0001:0000fe38       RegQueryValueExW           10010e38 f   coredll:COREDLL.dll
 0001:0000fe48       StringCchPrintfW           10010e48 f   coredll:COREDLL.dll
 0001:0000fe58       RegOpenKeyExW              10010e58 f   coredll:COREDLL.dll
 0001:0000fe68       StringCchCatW              10010e68 f   coredll:COREDLL.dll
 0001:0000fe78       LoadLibraryW               10010e78 f   coredll:COREDLL.dll
 0001:0000fe88       GetProcAddressW            10010e88 f   coredll:COREDLL.dll
 0001:0000fe98       RegEnumValueW              10010e98 f   coredll:COREDLL.dll
 0001:0000fea8       CeSafeCopyMemory           10010ea8 f   coredll:COREDLL.dll
 0001:0000feb8       RegDeleteKeyW              10010eb8 f   coredll:COREDLL.dll
 0001:0000fec8       RegSetValueExW             10010ec8 f   coredll:COREDLL.dll
 0001:0000fed8       RegCreateKeyExW            10010ed8 f   coredll:COREDLL.dll
 0001:0000fee8       StringCchLengthW           10010ee8 f   coredll:COREDLL.dll
 0001:0000fef8       DisableThreadLibraryCalls  10010ef8 f   coredll:COREDLL.dll
 0001:0000ff08       RegisterDbgZones           10010f08 f   coredll:COREDLL.dll
 0001:0000ff18       ProfileStop                10010f18 f   coredll:COREDLL.dll
 0001:0000ff28       ProfileStart               10010f28 f   coredll:COREDLL.dll
 0001:0000ff38       MmMapIoSpace               10010f38 f   ceddk:CEDDK.dll
 0001:0000ff48       DDKIomuxSetPadConfig       10010f48 f   cspddk:CSPDDK.dll
 0001:0000ff58       DDKIomuxSetPinMux          10010f58 f   cspddk:CSPDDK.dll
 0001:0000ff68       DDKClockGetGatingMode      10010f68 f   cspddk:CSPDDK.dll
 0001:0000ff78       DDKClockSetGatingMode      10010f78 f   cspddk:CSPDDK.dll
 0001:0000ff88       _DllMainCRTStartup         10010f88 f   corelib0:pegdmain.obj
 0001:00010120       __security_init_cookie     10011120 f   corelib0:seccinit.obj
 0001:000101b8       __GSHandlerCheck           100111b8 f   corelib0:gshandler.obj
 0001:000101fc       __GSHandlerCheckCommon     100111fc f   corelib0:gshandler.obj
 0001:000102a0       __security_check_cookie    100112a0 f   corelib0:armsecgs.obj
 0001:000102b0       __gsfailure                100112b0     corelib0:armsecgs.obj
 0001:000102f4       __GSHandlerCheck_SEH       100112f4 f   corelib0:gshandlerseh.obj
 0001:00010378       exit                       10011378 f   corelib0:cexit.obj
 0001:0001049c       _exit                      1001149c f   corelib0:cexit.obj
 0001:000104bc       _cexit                     100114bc f   corelib0:cexit.obj
 0001:000104d4       _c_exit                    100114d4 f   corelib0:cexit.obj
 0001:000104ec       _initterm                  100114ec f   corelib0:crt0dat.obj
 0001:00010538       _cinit                     10011538 f   corelib0:crt0dat.obj
 0001:00010568       __crt_ExitProcess          10011568 f   corelib0:exitproc_proxy.obj
 0001:00010594       GetCurrentProcess          10011594 f i corelib0:exitproc_proxy.obj
 0001:000105ac       _onexit                    100115ac f   corelib0:onexit.obj
 0001:00010788       atexit                     10011788 f   corelib0:onexit.obj
 0001:000107d8       memcpy                     100117d8 f   corelib1:COREDLL.dll
 0001:000107e8       memset                     100117e8 f   corelib1:COREDLL.dll
 0001:000107f8       towlower                   100117f8 f   corelib1:COREDLL.dll
 0001:00010808       __C_specific_handler       10011808 f   corelib1:COREDLL.dll
 0001:00010818       memcmp                     10011818 f   corelib1:COREDLL.dll
 0001:00010828       wcsstr                     10011828 f   corelib1:COREDLL.dll
 0001:00010838       wcstoul                    10011838 f   corelib1:COREDLL.dll
 0001:00010848       wcslen                     10011848 f   corelib1:COREDLL.dll
 0001:00010858       _wcsicmp                   10011858 f   corelib1:COREDLL.dll
 0001:00010868       _wcslwr_s                  10011868 f   corelib1:COREDLL.dll
 0001:00010878       wcsrchr                    10011878 f   corelib1:COREDLL.dll
 0001:00010888       wcsncmp                    10011888 f   corelib1:COREDLL.dll
 0001:00010898       _XcptFilter                10011898 f   corelib1:COREDLL.dll
 0001:000108a8       __security_gen_cookie2     100118a8 f   corelib1:COREDLL.dll
 0001:000108b8       __report_gsfailure         100118b8 f   corelib1:COREDLL.dll
 0001:000108c8       free                       100118c8 f   corelib1:COREDLL.dll
 0001:000108d8       realloc                    100118d8 f   corelib1:COREDLL.dll
 0001:000108e8       malloc                     100118e8 f   corelib1:COREDLL.dll
 0001:000108f8       _msize                     100118f8 f   corelib1:COREDLL.dll
 0001:00010908       ?CSPKppGetIrq@@YAIXZ       10011908 f   Keypad_mx25_topaz_v1:soc_keypad.obj
 0001:00010920       ?CSPKppGetBaseRegAddr@@YAIXZ 10011920 f   Keypad_mx25_topaz_v1:soc_keypad.obj
 0001:0001093c       TerminateProcess           1001193c f   coredll:COREDLL.dll
 0001:00010964       ?KPP_Entry@@YAHIP6AXIIH@ZPAPAUtagKEYBD_PDD@@@Z 10011964 f   Keypad_mx25_topaz_v1:kbd.obj
 0001:00010b04       ?KeybdPdd_PowerHandler@@YAXH@Z 10011b04 f   Keypad_mx25_topaz_v1:keypad.obj
 0001:00010ba4       ?KppIsrThreadProc@@YAHPAX@Z 10011ba4 f   Keypad_mx25_topaz_v1:keypad.obj
 0001:00010eac       ?KppIsrThreadStart@@YAHXZ  10011eac f   Keypad_mx25_topaz_v1:keypad.obj
 0001:00010fbc       ?KppInitialize@@YAHXZ      10011fbc f   Keypad_mx25_topaz_v1:keypad.obj
 0001:000112f4       ?KeybdIstLoop@@YAHPAUtagKEYBD_IST@@@Z 100122f4 f   KeybdIst:KeybdIst.obj
 0001:00011524       InterruptInitialize        10012524 f   coredll:COREDLL.dll
 0001:00011534       KernelIoControl            10012534 f   coredll:COREDLL.dll
 0001:00011544       InterruptDone              10012544 f   coredll:COREDLL.dll
 0001:0001161c       __IMPORT_DESCRIPTOR_COREDLL 1001261c     coredll:COREDLL.dll
 0001:00011630       __IMPORT_DESCRIPTOR_CEDDK  10012630     ceddk:CEDDK.dll
 0001:00011644       __IMPORT_DESCRIPTOR_CSPDDK 10012644     cspddk:CSPDDK.dll
 0001:00011658       __NULL_IMPORT_DESCRIPTOR   10012658     coredll:COREDLL.dll
 0002:00000000       __imp_MmMapIoSpace         10013000     ceddk:CEDDK.dll
 0002:00000004       \177CEDDK_NULL_THUNK_DATA  10013004     ceddk:CEDDK.dll
 0002:00000008       __imp_LeaveCriticalSection 10013008     coredll:COREDLL.dll
 0002:0000000c       __imp_GetTickCount         1001300c     coredll:COREDLL.dll
 0002:00000010       __imp_EnterCriticalSection 10013010     coredll:COREDLL.dll
 0002:00000014       __imp_InitializeCriticalSection 10013014     coredll:COREDLL.dll
 0002:00000018       __imp_DeviceIoControl      10013018     coredll:COREDLL.dll
 0002:0000001c       __imp_SetLastError         1001301c     coredll:COREDLL.dll
 0002:00000020       __imp_LocalFree            10013020     coredll:COREDLL.dll
 0002:00000024       __imp_FreeLibrary          10013024     coredll:COREDLL.dll
 0002:00000028       __imp_DeleteCriticalSection 10013028     coredll:COREDLL.dll
 0002:0000002c       __imp_CloseHandle          1001302c     coredll:COREDLL.dll
 0002:00000030       __imp_LocalAlloc           10013030     coredll:COREDLL.dll
 0002:00000034       __imp_CreateThread         10013034     coredll:COREDLL.dll
 0002:00000038       __imp_CreateEventW         10013038     coredll:COREDLL.dll
 0002:0000003c       __imp_WaitForSingleObject  1001303c     coredll:COREDLL.dll
 0002:00000040       __imp_SetThreadPriority    10013040     coredll:COREDLL.dll
 0002:00000044       __imp_EventModify          10013044     coredll:COREDLL.dll
 0002:00000048       __imp_keybd_eventEx        10013048     coredll:COREDLL.dll
 0002:0000004c       __imp_WaitForMultipleObjects 1001304c     coredll:COREDLL.dll
 0002:00000050       __imp_StopDeviceNotifications 10013050     coredll:COREDLL.dll
 0002:00000054       __imp_CreateFileW          10013054     coredll:COREDLL.dll
 0002:00000058       __imp_ReadMsgQueue         10013058     coredll:COREDLL.dll
 0002:0000005c       __imp_Sleep                1001305c     coredll:COREDLL.dll
 0002:00000060       __imp_GetLastError         10013060     coredll:COREDLL.dll
 0002:00000064       __imp_CreateMsgQueue       10013064     coredll:COREDLL.dll
 0002:00000068       __imp_StringCchCopyW       10013068     coredll:COREDLL.dll
 0002:0000006c       __imp_RegCloseKey          1001306c     coredll:COREDLL.dll
 0002:00000070       __imp_RegQueryValueExW     10013070     coredll:COREDLL.dll
 0002:00000074       __imp_StringCchPrintfW     10013074     coredll:COREDLL.dll
 0002:00000078       __imp_RegOpenKeyExW        10013078     coredll:COREDLL.dll
 0002:0000007c       __imp_StringCchCatW        1001307c     coredll:COREDLL.dll
 0002:00000080       __imp_LoadLibraryW         10013080     coredll:COREDLL.dll
 0002:00000084       __imp_GetProcAddressW      10013084     coredll:COREDLL.dll
 0002:00000088       __imp_RegEnumValueW        10013088     coredll:COREDLL.dll
 0002:0000008c       __imp_CeSafeCopyMemory     1001308c     coredll:COREDLL.dll
 0002:00000090       __imp_RegDeleteKeyW        10013090     coredll:COREDLL.dll
 0002:00000094       __imp_RegSetValueExW       10013094     coredll:COREDLL.dll
 0002:00000098       __imp_RegCreateKeyExW      10013098     coredll:COREDLL.dll
 0002:0000009c       __imp_StringCchLengthW     1001309c     coredll:COREDLL.dll
 0002:000000a0       __imp_DisableThreadLibraryCalls 100130a0     coredll:COREDLL.dll
 0002:000000a4       __imp_RegisterDbgZones     100130a4     coredll:COREDLL.dll
 0002:000000a8       __imp_ProfileStop          100130a8     coredll:COREDLL.dll
 0002:000000ac       __imp_ProfileStart         100130ac     coredll:COREDLL.dll
 0002:000000b0       __imp_RequestDeviceNotifications 100130b0     coredll:COREDLL.dll
 0002:000000b4       __imp_NKDbgPrintfW         100130b4     coredll:COREDLL.dll
 0002:000000b8       __imp_KernelIoControl      100130b8     coredll:COREDLL.dll
 0002:000000bc       __imp_InterruptInitialize  100130bc     coredll:COREDLL.dll
 0002:000000c0       __imp_TerminateProcess     100130c0     coredll:COREDLL.dll
 0002:000000c4       __imp__msize               100130c4     corelib1:COREDLL.dll
 0002:000000c8       __imp_malloc               100130c8     corelib1:COREDLL.dll
 0002:000000cc       __imp_memcpy               100130cc     corelib1:COREDLL.dll
 0002:000000d0       __imp_memset               100130d0     corelib1:COREDLL.dll
 0002:000000d4       __imp_towlower             100130d4     corelib1:COREDLL.dll
 0002:000000d8       __imp___C_specific_handler 100130d8     corelib1:COREDLL.dll
 0002:000000dc       __imp_memcmp               100130dc     corelib1:COREDLL.dll
 0002:000000e0       __imp___rt_udiv            100130e0     corelib1:COREDLL.dll
 0002:000000e4       __imp_wcsstr               100130e4     corelib1:COREDLL.dll
 0002:000000e8       __imp_wcstoul              100130e8     corelib1:COREDLL.dll
 0002:000000ec       __imp_wcslen               100130ec     corelib1:COREDLL.dll
 0002:000000f0       __imp__wcsicmp             100130f0     corelib1:COREDLL.dll
 0002:000000f4       __imp__wcslwr_s            100130f4     corelib1:COREDLL.dll
 0002:000000f8       __imp_wcsrchr              100130f8     corelib1:COREDLL.dll
 0002:000000fc       __imp_wcsncmp              100130fc     corelib1:COREDLL.dll
 0002:00000100       __imp__XcptFilter          10013100     corelib1:COREDLL.dll
 0002:00000104       __imp___security_gen_cookie2 10013104     corelib1:COREDLL.dll
 0002:00000108       __imp___report_gsfailure   10013108     corelib1:COREDLL.dll
 0002:0000010c       __imp_free                 1001310c     corelib1:COREDLL.dll
 0002:00000110       __imp_realloc              10013110     corelib1:COREDLL.dll
 0002:00000114       __imp_InterruptDone        10013114     coredll:COREDLL.dll
 0002:00000118       \177COREDLL_NULL_THUNK_DATA 10013118     coredll:COREDLL.dll
 0002:0000011c       __imp_DDKClockGetGatingMode 1001311c     cspddk:CSPDDK.dll
 0002:00000120       __imp_DDKIomuxSetPinMux    10013120     cspddk:CSPDDK.dll
 0002:00000124       __imp_DDKIomuxSetPadConfig 10013124     cspddk:CSPDDK.dll
 0002:00000128       __imp_DDKClockSetGatingMode 10013128     cspddk:CSPDDK.dll
 0002:0000012c       \177CSPDDK_NULL_THUNK_DATA 1001312c     cspddk:CSPDDK.dll
 0002:00000540       dpCurSettings              10013540     LayoutManager:Zones.obj
 0002:0000098c       __security_cookie          1001398c     corelib0:seccinit.obj
 0002:00000990       __security_cookie_complement 10013990     corelib0:seccinit.obj
 0002:00000994       ?g_rgpfnPddEntries@@3PAP6AHIP6AXIIH@ZPAPAUtagKEYBD_PDD@@@ZA 10013994     PddList_common_topaz_v1:pddlist.obj
 0002:00000af0       ?g_csEventCallback@@3UCRITICAL_SECTION@@A 10013af0     LayoutManager:LayMgr.obj
 0002:00000e4c       _exitflag                  10013e4c     corelib0:cexit.obj
 0002:00000e50       ?v_uiPddId@@3IA            10013e50     Keypad_mx25_topaz_v1:kbd.obj
 0002:00000e54       ?v_pfnKeybdEvent@@3P6AXIIH@ZA 10013e54     Keypad_mx25_topaz_v1:kbd.obj
 0002:00000e58       ?g_dwSysIntr_Keybd@@3KA    10013e58     Keypad_mx25_topaz_v1:keypad.obj
 0002:00000e5c       ?g_hevInterrupt@@3PAXA     10013e5c     Keypad_mx25_topaz_v1:keypad.obj
 0002:00000e64       ?g_fExiting@@3HC           10013e64     KeybdIst:KeybdIst.obj
 0002:00000e68       __onexitend                10013e68     <common>
 0002:00000e6c       __onexitbegin              10013e6c     <common>
 0002:00000e70       _pRawDllMain               10013e70     <common>

 entry point at        0001:0000ff88

 Static symbols

 0001:000040c4       ?KppScanSequence@@YAIQAIQAHH@Z 100050c4 f   BSPKeypad:bspkeypad.obj
 0001:00004fe4       ?KppSaveRegState@@YAXXZ    10005fe4 f   BSPKeypad:bspkeypad.obj
 0001:0000506c       ?KppRestoreRegState@@YAXXZ 1000606c f   BSPKeypad:bspkeypad.obj
 0001:00005150       ?KppBusyWait@@YAXK@Z       10006150 f   BSPKeypad:bspkeypad.obj
 0001:00005390       ?pKeybdPddInfoFromId@@YAPAUtagKEYBD_PDD_INFO@@I@Z 10006390 f   LayoutManager:LayMgr.obj
 0001:00005514       ?BroadcastToKeyboards@@YAHKPAXK@Z 10006514 f   LayoutManager:LayMgr.obj
 0001:00005c10       ?LockConfig@@YAXXZ         10006c10 f   LayoutManager:LayMgr.obj
 0001:00005c90       ?UnlockConfig@@YAXXZ       10006c90 f   LayoutManager:LayMgr.obj
 0001:00005d14       ?IsLocked@@YAHXZ           10006d14 f   LayoutManager:LayMgr.obj
 0001:00005d54       ?ValidateInputLanguage@@YAHPBU_INPUT_LANGUAGE@@@Z 10006d54 f   LayoutManager:LayMgr.obj
 0001:00005f50       ?VKeyToUnicode@@YAIPAUtagINPUT_LANGUAGE_INFO@@IIPAII@Z 10006f50 f   LayoutManager:LayMgr.obj
 0001:0000629c       ?GetModifierBits@@YAGPBUMODIFIERS@@PBUMODIFIER_TO_SHIFT@@I@Z 1000729c f   LayoutManager:LayMgr.obj
 0001:0000642c       ?GetModificationNumber@@YAGPBUMODIFIERS@@G@Z 1000742c f   LayoutManager:LayMgr.obj
 0001:00006510       ?SearchVkToWCharTables@@YAPBU_VK_TO_WCHARS1@@IPAPBU_VK_TO_WCHAR_TABLE@@@Z 10007510 f   LayoutManager:LayMgr.obj
 0001:00006780       ?ProcessModBitsForAttributes@@YAXKIPAGPAPBU_VK_TO_WCHARS1@@@Z 10007780 f   LayoutManager:LayMgr.obj
 0001:00006a70       ?GetCharacters@@YAIPAUtagINPUT_LANGUAGE_INFO@@PBU_VK_TO_WCHAR_TABLE@@PBU_VK_TO_WCHARS1@@GIPAII@Z 10007a70 f   LayoutManager:LayMgr.obj
 0001:00006f18       ?GetControlledChar@@YAGII@Z 10007f18 f   LayoutManager:LayMgr.obj
 0001:00006f8c       ?WriteToCharBuffer@@YAXGIPAI0@Z 10007f8c f   LayoutManager:LayMgr.obj
 0001:000070cc       ?ProcessDeadKeys@@YAIPAGPBU_DEADKEY@@GPAIII@Z 100080cc f   LayoutManager:LayMgr.obj
 0001:000073ac       ?ProcessLigature@@YAIPAUtagINPUT_LANGUAGE_INFO@@IIGPAII@Z 100083ac f   LayoutManager:LayMgr.obj
 0001:00007774       ?KeybdDriverKeyStateToShiftFlags@@YAXQBEIPBU_VK_TO_SHIFT@@1PAI@Z 10008774 f   LayoutManager:LayMgr.obj
 0001:00007960       ?MapLRVKeyToCommonVKey@@YAII@Z 10008960 f   LayoutManager:LayMgr.obj
 0001:000079ec       ?NewKeyStateFlags@@YAIII@Z 100089ec f   LayoutManager:LayMgr.obj
 0001:00007a98       ?AltNumKeyEvent@@YAHIIPAI0@Z 10008a98 f   LayoutManager:LayMgr.obj
 0001:00007ed8       ?AltNumOkToStart@@YAHI@Z   10008ed8 f   LayoutManager:LayMgr.obj
 0001:000082a4       ?ValidateDeviceLayout@@YAHPBUtagDEVICE_LAYOUT@@@Z 100092a4 f   LayoutManager:LayMgr.obj
 0001:000083d8       ?ScanCodeToVKey@@YAHIPAPAUScanCodeToVKeyData@@IPAI@Z 100093d8 f   LayoutManager:LayMgr.obj
 0001:00008754       ?VKeyToScanCode@@YAIIPBU_VKEY_TO_SCANCODE@@@Z 10009754 f   LayoutManager:LayMgr.obj
 0001:00008878       ?MapCommonVKeyToLVKey@@YAII@Z 10009878 f   LayoutManager:LayMgr.obj
 0001:00008bc8       ?pKeybdCallbacksFromId@@YAPAUtagKEYBD_CALLBACKS@@I@Z 10009bc8 f   LayoutManager:LayMgr.obj
 0001:00008c48       ?VKeyToUnicodeInfo@@YAXPAUKBDI_VKEY_TO_UNICODE_INFO@@@Z 10009c48 f   LayoutManager:LayMgr.obj
 0001:00008c74       ?BroadcastQueryToKeyboards@@YAHKPAXK@Z 10009c74 f   LayoutManager:LayMgr.obj
 0001:00009488       ?pKeybdPddFromId@@YAPAUtagKEYBD_PDD@@I@Z 1000a488 f   LayoutManager:LayMgr.obj
 0001:00009e68       ?pKeybdGUIDFromId@@YAQBU_GUID@@I@Z 1000ae68 f   LayoutManager:LayMgr.obj
 0001:00009e9c       ?ValidateKeybdPdd@@YAHPBUtagKEYBD_PDD@@@Z 1000ae9c f   LayoutManager:LayMgr.obj
 0001:00009ec0       ?KeybdEventThreadProc@@YAKPAX@Z 1000aec0 f   LayoutManager:LayMgr.obj
 0001:0000a620       ?pDLIFromPDDIndex@@YAPAUtagDEVICE_LAYOUT_INFO@@I@Z 1000b620 f   LayoutManager:LayMgr.obj
 0001:0000a6a0       ?SendRemappedEvent@@YAXIIIHPAUtagDEVICE_LAYOUT_INFO@@I@Z 1000b6a0 f   LayoutManager:LayMgr.obj
 0001:0000aaa8       ?Keybd_EventFlags@@YAKIIIH@Z 1000baa8 f   LayoutManager:LayMgr.obj
 0001:0000ab38       ?CallDLRemapFn@@YAIP6AIPBU_KEYBD_EVENT@@IPAU1@I@Z0I1I@Z 1000bb38 f   LayoutManager:LayMgr.obj
 0001:0000ac98       ?WillKeyUp@@YAHIPBUtagDEVICE_LAYOUT_INFO@@@Z 1000bc98 f   LayoutManager:LayMgr.obj
 0001:0000ad8c       ?KeybdEventCallback@@YAXIIH@Z 1000bd8c f   LayoutManager:LayMgr.obj
 0001:0000ae38       ?KbdNotificationThread@@YAKPAX@Z 1000be38 f   LayoutManager:LayMgr.obj
 0001:0000b718       ?SzToHkl@@YAPAUHKL__@@PBG@Z 1000c718 f   LayoutManager:LayMgr.obj
 0001:0000b838       ?GetDefaultInputMethodName@@YAHPAGE@Z 1000c838 f   LayoutManager:LayMgr.obj
 0001:0000bad8       ?GetPreloadInputMethodName@@YAHIPAGE@Z 1000cad8 f   LayoutManager:LayMgr.obj
 0001:0000bca0       ?GetPreloadInputMethodKey@@YAHIPAPAUHKEY__@@@Z 1000cca0 f   LayoutManager:LayMgr.obj
 0001:0000be8c       ?OpenKey@@YAHPAUHKEY__@@PBGPAPAU1@@Z 1000ce8c f   LayoutManager:LayMgr.obj
 0001:0000bf34       ?OpenPreloadKey@@YAHPAPAUHKEY__@@@Z 1000cf34 f   LayoutManager:LayMgr.obj
 0001:0000bfbc       ?GetPreloadUnNamedValue@@YAHPAGE@Z 1000cfbc f   LayoutManager:LayMgr.obj
 0001:0000c174       ?SetInputLanguage@@YAHPAUHKL__@@PAPAU1@@Z 1000d174 f   LayoutManager:LayMgr.obj
 0001:0000c84c       ?HklToSz@@YAPAGPAUHKL__@@QAG@Z 1000d84c f   LayoutManager:LayMgr.obj
 0001:0000c960       ?IsHklIme@@YAHPAUHKL__@@@Z 1000d960 f   LayoutManager:LayMgr.obj
 0001:0000c9a8       ?GetInputMethodInfo@@YAHPBGPAUtagINPUT_LANGUAGE_INFO@@@Z 1000d9a8 f   LayoutManager:LayMgr.obj
 0001:0000cd48       ?OpenKeyboardLayoutsKey@@YAHPAPAUHKEY__@@@Z 1000dd48 f   LayoutManager:LayMgr.obj
 0001:0000cdcc       ?GenerateModifierToShiftTable@@YAHPAUtagINPUT_LANGUAGE_INFO@@@Z 1000ddcc f   LayoutManager:LayMgr.obj
 0001:0000d0d4       ?FindVkToShift@@YAPBU_VK_TO_SHIFT@@EPBU1@@Z 1000e0d4 f   LayoutManager:LayMgr.obj
 0001:0000d194       ?GetImeKeyboardLayout@@YAPAUHKL__@@PAU1@@Z 1000e194 f   LayoutManager:LayMgr.obj
 0001:0000d40c       ?GetKeyboardProcAddr@@YAPAXPAUHINSTANCE__@@PBG@Z 1000e40c f   LayoutManager:LayMgr.obj
 0001:0000d548       ?SetDeviceLayout@@YAHPAUHKL__@@I@Z 1000e548 f   LayoutManager:LayMgr.obj
 0001:0000db10       ?GetDeviceLayoutEntry@@YAHPBG0PAPAUHINSTANCE__@@PAP6AHPAUtagDEVICE_LAYOUT@@@Z@Z 1000eb10 f   LayoutManager:LayMgr.obj
 0001:0000dd44       ?SelectDeviceLayout@@YAHQBGPBUtagKEYBD_PDD@@PAGK2K@Z 1000ed44 f   LayoutManager:LayMgr.obj
 0001:0000e1fc       ?DeviceLayoutMatchesPDD@@YAHPBG00GPAGK@Z 1000f1fc f   LayoutManager:LayMgr.obj
 0001:0000e634       ?FormDeviceLayoutEntry@@YAXPBG0PAGK@Z 1000f634 f   LayoutManager:LayMgr.obj
 0001:0000f450       ?IsLayoutLoaded@@YAHPBG@Z  10010450 f   LayoutManager:LayMgr.obj
 0001:0000f560       ?GetFirstOpenPreloadIndex@@YAHPAI@Z 10010560 f   LayoutManager:LayMgr.obj
 0001:0000ffd8       _DllMainCRTStartupHelper   10010fd8 f   corelib0:pegdmain.obj
 0001:00010398       doexit                     10011398 f   corelib0:cexit.obj
 0001:0001094c       ?KPP_PowerHandler@@YAXIH@Z 1001194c f   Keypad_mx25_topaz_v1:kbd.obj
 0001:00010c8c       ?KeybdPdd_GetEventEx2@@YAIIQAIQAH@Z 10011c8c f   Keypad_mx25_topaz_v1:keypad.obj
